:100000000C94A7130C94222F0C94FB2E0C94CF135A
:100010000C94CF130C94CF130C94CF130C94CF13D8
:100020000C94CF130C94CF130C94CF130C94CF13C8
:100030000C94CF130C94CF130C94CF130C94CF13B8
:100040000C94B12E0C94CF130C94CF130C94CF13AB
:100050000C94CF130C94CF130C94CF130C94CF1398
:100060000C94492F0C94CF130000000000000000F6
:100070000000000000000000000000000000000080
:100080000000000000000000002070702000000050
:100090000000000000000000000000000000000060
:1000A0000000000000000000000000000000000050
:1000B00000000000000000000000000000FEFDFB4A
:1000C000070707070707FBFDFE0000F7E3C1000075
:1000D00000000000C1E3F700003F5F6F70707070B8
:1000E00070706F5F3F000000000000000000000023
:1000F000F8FCFE0000000000000000000000C1E36A
:10010000F700000000000000000000000F1F3F008B
:1001100000000103070707070707FBFDFE0000F0CB
:10012000E8DC1C1C1C1C1C1C1D0B0700003F5F6F27
:10013000707070707070604000000000010307076D
:1001400007070707FBFDFE000000081C1C1C1C1C09
:100150001C1CDDEBF7000000406070707070707068
:100160006F5F3F0000FEFCF8000000000000F8FC9C
:10017000FE0000070B1D1C1C1C1C1C1CDDEBF700EB
:10018000000000000000000000000F1F3F0000FE04
:10019000FDFB0707070707070301000000070B1D0A
:1001A0001C1C1C1C1C1CDCE8F00000004060707073
:1001B000707070706F5F3F0000FEFDFB0707070760
:1001C00007070301000000F7EBDD1C1C1C1C1C1CB6
:1001D000DCE8F000003F5F6F7070707070706F5FF0
:1001E0003F0000000103070707070707FBFDFE00AC
:1001F00000000000000000000000C1E3F700000064
:1002000000000000000000000F1F3F0000FEFDFB8B
:10021000070707070707FBFDFE0000F7EBDD1C1CC7
:100220001C1C1C1CDDEBF700003F5F6F70707070D2
:1002300070706F5F3F0000FEFDFB070707070707B1
:10024000FBFDFE0000070B1D1C1C1C1C1C1CDDEB19
:10025000F700000040607070707070706F5F3F005A
:10026000000000000000000000000000000000008E
:10027000000000F0F0000000000000171700000070
:1002800000707000707000000000000000000000AE
:1002900040F0F040F0F04000041F1F041F1F040056
:1002A000E0F010FC103020000819117F111F0E0023
:1002B00060F0906080C06000000C06030D1E120C00
:1002C00000E0F01010302000000E1F11111F1E0062
:1002D000000000707000000000000000000000003E
:1002E000000000C0E0301000000000070F181000F0
:1002F000001030E0C00000000010180F07000000E0
:100300000060C0F0C06000000003010701030000AE
:10031000000000C0C000000000010107070101004B
:1003200000000000000000000000407030000000ED
:1003300000000000000000000000010101010000B9
:10034000000000000000000000000010100000008D
:1003500000000080F070000000001C1F030000007F
:1003600000E0F01090F0E000000F1F13111F0F00CD
:1003700000C060F0F00000000010101F1F101000FF
:100380000020301090F06000001C1E1311101000AF
:100390000020301010F0E00000081811111F0E00AE
:1003A000000080C060F0F00000030302021F1F0085
:1003B00000F0F0909090100000081810101F0F002F
:1003C00000E0F01010302000000F1F11111F0E0070
:1003D0000010101090F07000001C1E0301000000BF
:1003E00000E0F01010F0E000000E1F11111F0E00D1
:1003F00000E0F01010F0E00000081911111F0F00CC
:10040000000000404000000000000010100000004C
:10041000000000404000000000004070300000007C
:1004200000000080C040000000000103060400003E
:1004300000008080808000000000020202020000B4
:10044000000040C08000000000000406030100001E
:100450000020301090F0600000000017170000002E
:10046000E0109050D010E0000F1013141714030088
:1004700000E0F01010F0E000001F1F02021F1F003C
:1004800000F0F01010F0E000001F1F11111F0E000F
:1004900000E0F01010302000000F1F1010180800AE
:1004A00000F0F01010F0E000001F1F10101F0F00F0
:1004B00000F0F01010101000001F1F11111010009C
:1004C00000F0F01010101000001F1F0101000000CC
:1004D00000E0F01010302000000F1F10111F1F004F
:1004E00000F0F00000F0F000001F1F01011F1F00CE
:1004F000001010F0F01010000010101F1F1010005E
:100500000000001010F0F01000081810101F0F006D
:1005100000F0F080C0703000001F1F03061C1800A0
:1005200000F0F00000000000001F1F10101010006D
:10053000F0F0C080C0F0F0001F1F0001001F1F007E
:1005400000F0F08000F0F000001F1F01031F1F00EB
:1005500000E0F01010F0E000000F1F10101F0F005F
:1005600000F0F01010F0E000001F1F01010100007A
:1005700000E0F01010F0E000000F1F160C1F170035
:1005800000F0F01010F0E000001F1F03071D18001E
:1005900000E0F0101030200000081911111F0E00AB
:1005A000001010F0F01010000000001F1F000000ED
:1005B00000F0F00000F0F000000F1F10101F0F00FF
:1005C00000F0F00000F0F00000070F18180F07000F
:1005D000F0F000C000F0F0000F1F100F101F0F0010
:1005E0000070F08080F07000001C1E03031E1C00D1
:1005F0000070F08080F070000000001F1F000000FD
:100600000010101090F07000001C1E13111010004C
:10061000000000F0F01010000000001F1F1010007C
:10062000000070F080000000000000031F1C0000AC
:10063000001010F0F00000000010101F1F0000005C
:1006400000C060303060C00000000000000000000A
:10065000000000000000000040404040404040409A
:10066000000010302000000000000000000000002A
:100670000080C04040C08000000C1E12121F1F00EE
:1006800000F0F04040C08000001F1F10101F0F003E
:100690000080C04040C08000000F1F1010180800EC
:1006A0000080C04040F0F000000F1F10101F1F001E
:1006B0000080C04040C08000000F1F12121B0B00C2
:1006C000000080E0F09090000000001F1F0000007C
:1006D0000080C04040C0C00000276F48487F3F00F6
:1006E00000F0F04040C08000001F1F00001F1F00EE
:1006F000004040D0D00000000010101F1F1010005C
:100700000000004040D0D00000206040407F3F000B
:1007100000F0F00080C04000001F1F070D181000FF
:10072000001010F0F00000000010101F1F1010004B
:10073000C0C0408040C080001F1F0007001F1F0076
:1007400000C0C04040C08000001F1F00001F1F00ED
:100750000080C04040C08000000F1F10101F0F001D
:1007600000C0C04040C08000007F7F10101F0F00FD
:100770000080C04040C0C000000F1F10107F7F00ED
:1007800000C0C00080C0C000001F1F0100000000AA
:100790000080C04040C0800000091B12121E0C00E7
:1007A000000040E0E04040000000000F1F1010007B
:1007B00000C0C00000C0C000000F1F10101F0F00BD
:1007C00000C0C00000C0C00000070F18180F0700CD
:1007D000C0C0000000C0C0000F1F100F101F0F008E
:1007E00000C0C00000C0C00000181D07071D180091
:1007F00000C0C00000C0C00000276F48487F3F0015
:100800000040404040C0C00000181C1613111000EA
:10081000000000E0F01010000000010F1E1010009A
:10082000000000F0F00000000000001F1F000000AA
:10083000001010F0E00000000010101E0F0100007A
:1008400020301030203010000000000000000000B8
:10085000000080007301760178017A017C017F013C
:1008600081018401860188018A018C018E01900139
:1008700092019401510268028A029502F502650311
:1008800068039303AE03B103B403D903E203E703A0
:10089000EA03EC03EF03F203F503F703FB03FE03A4
:1008A000100427042D0432043404360439043C04B3
:1008B00040044304450449044B044E04500400031F
:1008C000740BD484606FAE6CF9BB84A265B14BF637
:1008D00072011A21E85AD8D604735E2C226EC4E93C
:1008E000B58B819A1EE487C99E7B17526DADE3E5F7
:1008F0008B04A72E996A32AA9997CCA65B157956D4
:10090000480163B1DF5427065706538CA627AA6611
:10091000890318517EFB67D3CEDD3FFD3D1F478421
:1009200001F3856EF83B792B0C904B67467D54881C
:10093000FDD612E5E748F20EDB994D71A54068D966
:10094000C95939E475201CE9B1F5013C19BB60F7C0
:10095000FA6B1E689F19B6ED140F56BCC134CB005C
:100960009D43D40FF3629C9DF78B9D533A8D2F3D91
:10097000DE3D3831039BC7C159E9D175888D3658A2
:1009800086704E5B9ED0DBCBF7EA1FDBA53BB3BD89
:100990006BBCF37065D5170F64152420D5B87B0D9B
:1009A000272985881F5822574F09C04DD6E4C6B560
:1009B0003A373327BB6A1469031BEDA8C343E8EA3F
:1009C000DE410625C5C83CBF32B2A7DD22C2E9CA56
:1009D00084F2C0267C7801F7D5C60533E4C278ECF2
:1009E0001BFDD2507D11295799B0F1556674B4584A
:1009F00023A06F2ED89B08B33E53CF5ECC7ADF4E38
:100A0000ED42166A9188431B1D845C52216658246E
:100A10003671C56A0D2C869A239DE03543C97F4106
:100A2000BD8299ED7A26B2D3A6CE4F00E687E3D7F2
:100A3000682886F7CED2B3D31B0402B978B3ADE0F1
:100A40003C53A68A4A22BE1FCEB176F22F81A8C19E
:100A50007872B0156519E332A74D0CD300B9C327DE
:100A6000BE744DD1E10C36DD23FBA722D344CAB3BB
:100A7000081BB40D4BDF1AA69032925C1AA7CD85E5
:100A80002E351172F821357D3FDB298D30B34F456E
:100A90001477CF992FA39081B0AEE845E63AA9A28A
:100AA00062B7DBBE2539A5FCEAC5BC3AEC90AEA620
:100AB000FB12AAC76222AFA984B964B8FB8DC11C1E
:100AC000C3D0876D5CB4FE3FA4B8D889F40159BB8C
:100AD00004A543441ACB4130F75B9AEE28F44C71DD
:100AE00099CA4B7F2A13F04B54B3FC90EDBE483F9C
:100AF000F15E0DA1BB1E591615F04B504C96861B8E
:100B0000A9CCC2694E1003F0E953E5E2BB45E28D82
:100B1000AE407108864D08F49690585340A58B5B03
:100B20003CAD47B5D7E26A1378D4DCC9EC0E93F03C
:100B3000C01D953676A45385C9ACE4718DAF68614C
:100B4000209DFF45356E04D82732C3DAEEA2660435
:100B5000B72106527F398FFDEE9074B64FB6240E42
:100B60001248F0B230F2A54C9152E3C6487B389659
:100B7000239ED71B95153AC98B6F637D1DC9EA96D5
:100B8000E601D785C0EA3DCAD3B7FB07543A003126
:100B90003D74E4125BA238335BBF1DDC4EE8851068
:100BA00077ABEA6579B0AA3061C6F63BCC95FC8399
:100BB0007F8C7BB55205EBF721DE89B66DEE317780
:100BC00013AA935596086E1C82B57E95B994DD687C
:100BD000425C3A00C37B6F606A2C07D76C82FBB221
:100BE000812569D6720AD2E8500588491B6372993B
:100BF0006CE37AAEB01B9ED42554258A901797DFFC
:100C000039B87CEAF082DD25D2ADE7F6362384A937
:100C1000C96A53F4822C1DEA06C64F705437802AE5
:100C20006B63DBCC86E68C7F278C7254739E1BD65D
:100C30004CFA058280D7B71198000000000000062A
:100C40009869151CFC868774845BD40FDBD727C595
:100C50004AB28F297A4A230AB807D03470818E535A
:100C6000EF43163FA8A79E5A77C091B789155248FF
:100C7000C0B762ABE1746410AA096B97742179352F
:100C8000A19725FC78C1EC6E877740871A74828122
:100C900056DDEC37ADAF0331AC478574C02A459DB6
:100CA000F4120CF986B04A16D8116C46C44A6798FB
:100CB0008B1B42C2BEBB0E4884F708A6C38F8E8D25
:100CC000ABC29B5D5C6028578F0EAD2EC15E95292F
:100CD0009AF48A27D441BB4AAC5DB29326FD878142
:100CE0003F2735A6422C1538ADF8026F94DA08EE8E
:100CF00019D890FA89C3AD89FEC60246811D0C8DB4
:100D0000782FEED3ED6C7B95495687F4E263DA39A0
:100D1000CE681618ED98EE86F3B3C1121A519B57A0
:100D20001D199E987ED2FD3D2B5915467457791496
:100D3000817189D922DD9210D98991DF67006E53C4
:100D4000AFDAB528301E47E6B7052D22CF7F6ACD32
:100D500088906B8C16368807A1B7AFF331C4DB7669
:100D60008B969EF017A73F847891A8CD3F8FA5DD85
:100D70005214F9395D0B568E1C5A5B89EE809E33F6
:100D8000BDB145154234597820FC2DDBC92E0F35F5
:100D900026CF239B3E1D9F0F260EB7B54EACA286D5
:100DA000D5DA36045A73466A88C52AA083E88B5F71
:100DB0003CAF6A444E759B8F93373538BD029A1D00
:100DC0008429642597E07C2AB6CBC166513CBC3BA4
:100DD000F3552BB7BD81ECF349D5F803E0BDC60C44
:100DE000EEC01908FB4F8C94080EA53037F0B818E8
:100DF000937300BB5252B4980D4B45B9890A34E93C
:100E00001C245A8FA89DC2D927A9EEBFC08090BCD0
:100E10002A9343FB0AB396D1AE13410168B92C5310
:100E2000537C00A58441D6988898FEDEF7E23743CC
:100E3000620E9383EE030A8DCA8759366F61F7F409
:100E4000D6AB8B0F9C8396A46C4643806BEA50DC38
:100E5000D8CED4F4AE5BC6014385718D0C395EE407
:100E60003B2BC488B2C554960E879A5093D69C915A
:100E7000CA09648B23C429441A67E1DAC71B251702
:100E8000022C8F2A133ACFD665312B10F5B596DF99
:100E900001997BADD6B4C035A348E3B09EFE3310B4
:100EA0001A09AE3C0AA1728F0051E17823F5E2BF26
:100EB000A64628B34B24B1A1DEB1C4486FED5AD485
:100EC00061F0DBE1085C64C0CAE9A9DEDEECC06861
:100ED0005B6DBD43828CCA69B1A9C8710D5D6DA5FA
:100EE000AB1A6794EE0593E33FE81AE60F7F79F2B9
:100EF000CBC53757DFFC4FB460C7973C61B00C4699
:100F000064F44392D2A5F0F3B7DFAB20B1F5302AF9
:100F1000B3DC4B39B7853E1E1B948C26288045D602
:100F20000136D0EC934688D3D5895D7A82213EC2C2
:100F300040E3B4DEF5A569D569495C89CDAE13708F
:100F400070ED690CECC6FE75EB4ED6B3C860FB3491
:100F50001EF86492D929A813383D79C4BF21379D62
:100F6000E34F21E53F2C5C5F41FF148791E0820451
:100F70000B1E5553DC5640A43578E29B49222E09BE
:100F8000CD1F6F9483EEEA8BC4C210E080D9A55FB9
:100F900053349C8CEA95648794D6321CEB93BFE360
:100FA0005583C2F6FCC885B2945C425F6B8E3B975A
:100FB00079747EE35CC2631A22B17F94CBE7B7FFFA
:100FC0000E3795AF105317881272DDCBAB4B6B68A1
:100FD00024ACC95C72094FF1FB1DE7A230E9204B3C
:100FE000DA707C9EE234EB6A35C233D79D07B1EFED
:100FF000F675F5FDADC74BD0B7DDAE1E8D1EC03901
:101000009CA71CC5CC3950C66BC6DA37C7E120EBAC
:1010100074A53DC008FAC2DFF29E432BF077504919
:101020008CC32F68F32A9B831ADC05D8B77C3C61FC
:101030001176EC2DFE86088715A3C01CB46A8D9E20
:10104000BF9AD5C85B05181015FBC63CEEC5524BC0
:10105000313607B94C81EA83D782FEFC43594E20D2
:10106000BDD365CF1F5C711FBF26EC44EB017482BA
:101070003C8E60DF479031177E16C0EC1EC33A7A73
:101080005921A29B8E8725D3FE85DD6DE6D8CA74D3
:10109000BADB4230963D8622866FDE371A932F03E5
:1010A0002EE16E1662C1E12DFECBA8DF6405EF23B1
:1010B000BC71617B1B602227BDC6A37207AA09B061
:1010C00052F219154DBEAF263B4D62A63C41077A40
:1010D00034253CD6CDB65547871ECBCFCED20D9505
:1010E000C0D872A6E0332426517E71C7533FD4671F
:1010F0007352CB785A001115715F8D3CCF40CDD91A
:101100007430D9A13FC658BCBE7818319A3960BB3B
:101110008D7B3495A5F1543BB98599AFC445EB64FB
:10112000A76E5960EB1E7AFBFD924323F127AC6654
:101130001266288A5CF6C63F7604E80927ED05AA00
:1011400026E5B4AD40BAF7F484CB7F07108DB6C75F
:10115000D477EABA962A98F056D7FF504D59793D80
:1011600041E0FAA99D3EA6D979C80DD156C5ADD7A3
:10117000FB703CBDF3E95D1C5393331DF81BEE9FE0
:10118000B750AC8F485961C9859EC8B0D27439DF59
:1011900033F528E06311A7C405BD3AD934CAF9AACA
:1011A000E200E6E638573EEC197C0D2745C552C4EF
:1011B000FFF469C5F573734FE307C7CF38235B9C12
:1011C00099A26A72B03539C10AC71C1A3060181D5D
:1011D0002BF0C8F179A394E3363593690591071292
:1011E0006044FDB6C6FFE0CFA2CFC2A358AC32E345
:1011F0002EEC0D9D1BFB0540BA678ECB38D7609C4B
:10120000FE9EA170CC40728C8C507185DD84925C06
:10121000EE44B6E0801532DD1B4B8C6E8E3997A5FF
:10122000AFC6F42985D3859385C854E4591D4EA0D3
:10123000FEC507C1F73252F94D4585FCA0FA37B516
:101240009D47E852238D928743B4B84F951B1E4F9C
:10125000E545BFCEC80CB27DE7D92E88B72A61E13B
:101260002DC4212EB84DFD2187302511EC1F299466
:1012700031D292853817DA634D8CB4065564B76C59
:10128000FCC28D5D978609D34369E83577CCAF9171
:10129000363C7CA36E4E4AA2C94150EAABDF8704BC
:1012A000704F16F5A038F56016CD0CE5C7E3AD001C
:1012B000126B12853C5C7F76ED49F29D8FDFABE1CE
:1012C000DD8701ED2C1B4B55117FC392D391C1D803
:1012D000A737C7E55B482BED31DECEFB950000005C
:1012E000000000000008E35184000B4D2673118BB1
:1012F0001EE20000000000000000040473E072FF22
:10130000E659C900000000000448BFABF399877C90
:1013100007000000000004FB33B163616112AD00FF
:101320000000000008AA30AC174D3086BF6713F1EB
:10133000A70000000000000000041B48422384BBFB
:101340007FB4000000000008A69F43785CA14E8B8C
:10135000A6E67C49000000000000000001F7315DB6
:1013600027300000000000000000010B570B79F748
:101370000000000000000000024433BBB45BC70063
:1013800000000000000001ABE301C2D20000000039
:1013900000000000017A079EAD84000000000000FC
:1013A000000002F1EEF7D829500000000000000014
:1013B000012C35543ACC000000000000000001C9A7
:1013C0003D666A980000000000000005247AF71CC2
:1013D0002440EBA24DC266C8372C030FF301066D03
:1013E0009A42F0948FEDBFE3283B72693775B4A041
:1013F0009A6E31FD665BCBF3BA8CA431FFBA7C24C4
:1014000054D3C6638993E4EDDA58474EB58FD7932A
:10141000FDAF31EAB4ECC9057D2B1596C1007E8085
:10142000E6F747CD6A77F10E5913AA5C838870DC22
:10143000C4525220B6692D6C6C8B662ACD5A41304D
:10144000D6FB7BA0EC7A22887C716EAF6206F4A892
:10145000C688857636C5C0D867967CE84DD4FBA98A
:101460006F0FB2A7A3196A30FD6FFC2BCEA41B8EA1
:10147000574851C6980FE5087B4DFC59DDCF131B2B
:10148000310C5E3B98E1F4C341D7A2645E16F9EBE0
:10149000AE20E95D54BD99D3A7C1D9E53222D69FCC
:1014A0004FDD6B3C6DE94D965211DA2386BE01C4C7
:1014B00051C29CC6F52F1FD0F1F55782FECBFB4AD7
:1014C000DF1D0046B8A73A566608714E47F8272632
:1014D0005F6CD8C305990A758F4FC18872A05A13E3
:1014E00008A382842ECEB5A34605D66A7856442337
:1014F00086F2C963088BBDEE56D4361F375318E702
:10150000DA1CFAD005D55FE7B7AD362BCB06C05352
:10151000F432A8756FE3C9A1B0A6E6C2410F5D2EF3
:101520000A64504692495B2D002EB5213F0B4A714B
:101530009688844C98AA2823EBEF455C6278D6E421
:10154000FB6DC3D9356CB92AC67471C40C657CA314
:10155000F96E2DB986B0046394CF267D9E1EF7994F
:10156000DAE08CDD86F3C8F1C64E155DED34BB9034
:10157000CDD626091EF6238451C1AE428F8496C96A
:1015800057AE16363A298765B2BA5696D2F509EFA4
:10159000304A0F6236FE0030BD091B50C33C48D7AD
:1015A00025E18EB26F4D752DADC61EBAFA4F41AF13
:1015B0007A6FA0A04FB68834698A9E837A60F3A8B8
:1015C0007E392A209C325E7DC4AA97E6263542A148
:1015D000A0EF39B31C2763D27F75C01EB4FA4D7AD1
:1015E000818139E0792F94A5283A437E97B594AF4D
:1015F0002A10380A7F4991C06C659AC6C95DD552D8
:10160000469874AC93E421B0EB08FAF4412EA6F9A5
:10161000C5EDE33798C5DF528241A2F2561AF3A412
:10162000C6408DB95FAA751E151E68782B2BF43E37
:10163000C7CBF31360E0F48579880C227587B75126
:10164000E0D6E3A092D3D7E36C5B3EB780E748D601
:10165000D92F49CC75A004C94888E9CC3241AF30B4
:10166000DEC6BC9DF7FCFF69035058A1D6B87B5E6F
:1016700060FCCC0014AF3A3041B34E634795E4BDF3
:101680005374D0F002B4FE48196C3F23F79B441109
:10169000F2C245A637776C10630E1BA7D196CA0D10
:1016A0004F5B4351D614B723E799A49F4C7DD7DDF8
:1016B0000811844D5CE96090048B1490F06F26450E
:1016C0000F208CE36F4678EB12B45EF0DEEB22273E
:1016D00062784293BCE848C088BD0FDE232BD188D6
:1016E0000AE2B4338E6136435842AE6BD7F2FE0A3B
:1016F000C126947ACE8C3B435A62EF708AFE4DD25B
:1017000037DBA1B1061B30174CA0241EBECB64E210
:10171000CE135CD705A6763938F3852C160EB3E2C6
:101720003DFF79880B93EFAD55CDB4EF8FB8167AA6
:1017300005C05E920F4F9858D422AD4325317852A0
:10174000C69ACA5EA64E79979ABBDF6DF1E2D0B316
:10175000CA2A5C46825C1EDDD0C519892B2CBDC00F
:1017600084D9333967E4E47926B69D1C1DE470A55D
:10177000A76189254A57337D0DCAF3CC22AAD7D950
:10178000CBE6B29646159568D80FDF6B36DA19822C
:1017900016CE384ECFF236C880075388042FB214C5
:1017A000195DC56CEF959C608B6AE4FC9DB29CED65
:1017B0001D9C1BCAA326DD9C635B3B882BBA22358C
:1017C000240148EEA04F6E964E2991AAAF5647BD10
:1017D0007BDDA15599D8B5A147937BCD7BCF65DE45
:1017E0005018F20549F199D894213F7D52C6B1B401
:1017F000E19FF07E60648B30E4AD2C97FB47F709E6
:1018000001047BF4F7A7A804A57F0858796D262763
:101810006AD0D9AFC1C71223E1AE98A40FBC1BFA9E
:101820009D910B1515A524531A13E0C30095389C00
:10183000364CCFF6A9BCC1530604F46FBF57E0A6DF
:1018400014A649707F392A4A5A593633B90D4725AB
:10185000393704777C45AC19932549E07A7BA2C6D9
:1018600095768D3C79B1A7C38363032347D7ACFB3F
:1018700084166F22490B97AAD538575E2BBBA74910
:10188000EDD2D57A96BE8DF5F94656F52FA7A87AF2
:10189000FF3FE7E88CF148E846CB4D25F935932F1B
:1018A000CE8BB8A9C5D3D22771866F72D9CA4E9094
:1018B000D36DB13CD3CBC9303A26459D66445C5FBD
:1018C000D8E3907C1BD882DDD384D4C61B58BF02DA
:1018D000A53B100A3EE309940B99882B47A79089F2
:1018E000C4482536DB7231ACF5A30115D0E6216181
:1018F000EB5972DC94000098F7B0F9FAC10A7EDC6B
:1019000069CE905E82110B97E29955A23DFAEB8861
:10191000BC4DC2548D5FDEA3E248132046C5A081B2
:1019200004C42B9A8415B89E9B62A1EC7D083CAD43
:10193000214B89FCC6967C3A41358A13BD1B43BFB7
:10194000367A4ECE709E2AF63933C7334B347D2A11
:1019500081FA252EC5C4A1280ED54D15E069127156
:1019600019AAFF5948815653C935124D84699136D9
:10197000D8ADF754D58CF9C684126222F1B92B1D6B
:10198000A57C567A4D5AC4F09D8F5DB59A7FE7B716
:10199000A85D6D3700000000E4F2EA7A73F8FC6796
:1019A00017F3D960090E8B0FE2F98361DF5369D019
:1019B000EE4251B5514864F8DD3EEEA747F07C4B4E
:1019C000BB2B8EE28B6057634B9BAA6763EAA3D560
:1019D0007C4341A95474D286C3114269C5093E8F24
:1019E00094AFC599BBBBAC61646101F2D359B141FD
:1019F0005091166CCC9BEC5CFE3BB3EC6ED7F10EB9
:101A00005A8A5F1DB0C576542607BC66F0ED519A20
:101A10001FE8F751588E1E80991FEED643CCFA2F3F
:101A2000AE80F2A8A8AE437C8076D41AD4737461D9
:101A3000DFBF296F561593075892F11DE87B68B2F6
:101A4000542030012DC5D8FD6150140F584C1A5444
:101A500000127E46990C9DD1A304F18217FEFC1260
:101A6000E57581AFFF3D08D539874A8EF07AD4D02D
:101A7000D6CFA9D6594841C268E3A435458D141A7A
:101A8000C4000000000044892C63C8AF7BAC354320
:101A900027BE7ECF56403DA5AC0F97CCD46ED0313B
:101AA000D7146045AEDF0AAA33B388E01C26DC00F9
:101AB000B875C86711A1B58771F94A6AEC3F0E4144
:101AC00021C24F928F1753EED5EA4F9175025900FC
:101AD00000000294E4DA4AB3AAA72E9CC780465EAF
:101AE000BD06331DD85D9F5F77730A7D386BA70EE7
:101AF0008F4E7D01DA4474D2F17A2F7FE1ECF1A5AB
:101B00007D033B2F17B6E80D333C2191915B302CC0
:101B100011C6586AE4351BB5A847B3FFD0960E48E6
:101B20004E9737601204FFCBA5F51D409CDF36129F
:101B30003DD92A72DAE88BE45BCFE93852EC2CA06D
:101B4000F779AD2070592062739CE34609C912D41D
:101B50007755074B6A261E5D0778104E4ADA5EF607
:101B60003B9B8DFD48D0BBAA212EF5DF854CA71DE0
:101B70001A261BA082867F4B02D2F660C9860C1DF6
:101B8000BF736986184B44BC74E5821793B50A5637
:101B900008B74A73B804D214215E2CA0E0C2015FDA
:101BA000DECE642AD8652BF074E354BFA09B50BAF4
:101BB00002002C95CE2A4FCF2B2B0E9BDD8F675B1F
:101BC00054A1472E842E24FA34E05A103BCFAFE2C2
:101BD000ED28D1176B9A1B496CFCCB7A74092A410A
:101BE0005AFFA1F598C60CD26983D2C369875E7E7D
:101BF000BBFCC0D1C117D79BE15370B743D0382588
:101C00002649405B57BA4932AA9F39AA8E7300858C
:101C100013796DF1912F9EA3A0657C7D53B4705311
:101C2000016B925F38F1D73D7AD607727ADBA165F6
:101C3000A50741004BEBC5D03BEB3061420D4BA3F8
:101C4000D8078B12F5893D7CFB2E79A7BCD5BF72D6
:101C50009AD81539AD2570D16CB05DBBF43AF660F9
:101C600056FAF2A528AE0D76B379F14BC72E6EB6B3
:101C7000616222D9A730234521DE478CEBE54C8BEE
:101C80004E79A09D95B305AAAFECE67473F0DC37EE
:101C9000AD933B206DA1D8CFF97E9EC6BB40645664
:101CA000A6187528D2BA78645C484570358C499A74
:101CB000454A6DF29C8D480A612EE3D4EEA8294076
:101CC0004B53BB5639CE816CFD37A0791CC7941796
:101CD0006C37EA97F4D8D49F9F304FE5A408B86BCF
:101CE000AEB9BC4F612044DF92DB1E0483C0A12C3F
:101CF00009D8DF21F0200480AF7391BC0EBAE4F75D
:101D00009B363C30F1B4BADCFA65F22B1D184E1646
:101D100062D4AC8B21A5A2F132C3C965632D316BAE
:101D2000B88FE12493870499E6BDBA283063DAAC12
:101D3000C799378A8666B344D584AAA15342A0388E
:101D40001E5DF70529E7CA2A0B6AABCEF03AF3907D
:101D5000E6D125A1331C33997D24D17423FC6F7DFA
:101D6000DBA7E9C2DE17122D1CB37E88000000003D
:101D700000000308757D9A4937AF60047CBCD31C12
:101D800053703497EBE1CD3079A28694585A99C2BA
:101D900069D7B232626C0A3669B1354841CE79965C
:101DA0007A0D2D33BF4D2FB8D8B3FBE47193B9181A
:101DB0000D51ABBB09D90DD7671E4728C7F7CE60B9
:101DC0005828235E95FC2BDBF90D1FAB49E6D0A705
:101DD000377920E4CF05E36421ACDFB1E8F9E04CCA
:101DE0003B5E89682A48C5640EDBF1538B1A2FF6D7
:101DF0000C189C529B212E4AE7D6BBB71A0A22AB7D
:101E00004AFDD3027D21FFB90E0F29ABACF4445E2D
:101E10000FD5F357E54F61724EBA55378F9A1CD4E0
:101E2000B830AF0A951A1386D40A835C991B2BC06D
:101E300093F513F5EAFB6F75746C2E77C344C538C0
:101E400062B9F5AC58B4966EA4A545B51B7C9D212E
:101E50009516EE29572012BBF80A2325AC51FD7ABE
:101E6000E09D43B0276F2ADF0408D3F11D3C128D9B
:101E7000AFF2D7B9029D46E3ABFF61C8612B19C829
:101E8000C1A16D0AA744FAB5A8D71E53156F7A48A9
:101E900041E930B5ADE2F070406AF331DD1950E54B
:101EA000BCB43D839FDFC8252790405B3204478147
:101EB000FA53B40A40157A745BDB24AB3AB791E36A
:101EC00044B747073990D2F5A9084658DC3210A329
:101ED00047320445441371AC2EA7C971D0F9517E25
:101EE000CAE509A81E775B3A08AA431CD68D609103
:101EF000466D64569E162ECEB399C8F655271384A8
:101F0000BC8AB3C8F51A72F76A0C46952F4A86B692
:101F1000D29894F1C3370E0C8711567EAFDA22297E
:101F20006FEBFAEC96E0276B42A170091AAD488876
:101F3000DAFCE13B62952856702803B258678D0A97
:101F4000EA9A1595515F83070920BF37AFF70A74E6
:101F50003CA552F1E3F55830E117DE98F1387BF0FB
:101F6000AFBD165952996C7470487714FF53418471
:101F7000BCC5372F71843DF5467C63E000A0560751
:101F8000F78C6357BE545CE1FDAC35FAC2D5F25A0A
:101F9000BE7C318EBDDBFE4D036F5EA61F232DCAB6
:101FA00068F0C614CCC33EF021D4402A72B67EE25B
:101FB00085D68AFB48512777E4CBCD2FF6E1BCFECE
:101FC000EDA1145FE532FCCFD9FB2FE9AD7D2D6883
:101FD000E79A15956A4AE4ABE4EBE00D40BDEF8F5C
:101FE000B975B439086DC09F04FFCCDE13304EB60E
:101FF000E4E0CB69E5C61C2F436A632572D5DFBDDB
:10200000DC0BE9089D3D266FC389F818AC42BF4E32
:102010009D5D28B0264136768D8684FAD8D46758DF
:102020001969202D35FE09D98CFDF921A157DF173B
:10203000AE8ECBC97F2654DE104372DDBC18B93496
:10204000F9AB70F9744D8E6D2A331406D071E6AD7C
:10205000AABE862E9A8D8788AF039FCBF8789A66A2
:102060003809CDAE89C2CCAF6A16140948AE9B556B
:10207000E40FA586A1757F7CEF0DCB3AB30D1F024F
:102080000000000C801FB4F4E0A641CC8700406142
:1020900043E7FCB40000000124CA4534253C39FF65
:1020A000098C39855A5BCC273CBD28438645179A55
:1020B0004E3524A423A2FDCA6CD4FBBAE741B3FB7E
:1020C0007C5507B56E3EB12972CC38EA273080B90D
:1020D0008CB8EE54AB3EDBDD06D095EA3E42886B11
:1020E000AE89C7E84C38B693F6BE4C204A8CCE2B4E
:1020F00022D272494618568070675AFAC0CA6D5388
:1021000021CAE3866891D37CA9D5AD6A72A1FE533A
:10211000E94085EA62A963753A2DEC9BFE58D873B5
:10212000205210435C2DB421B9961F726DBA42EA59
:10213000F285BE5212A7B13E2B89EF0F73057C9931
:10214000C3C55F9653F8AF9B7A49A044546055F0DD
:10215000103A608D905065AEF779DB2E08F9BBF22E
:10216000D278D086B594A10EB98189B7F9C043E879
:102170008F3819DAED2FA75CDB01B338CEE6C3F256
:10218000D5AA879E116FD805F072ABD9A10FFF4673
:10219000E94A8C0093E9866F6B1470BEB1B889C9A7
:1021A000CC7D1A11D279FBD9D72413948F019C4B83
:1021B00069336601829888F84C13310F58C10611B3
:1021C0003000000000B48991349B89FC75CD11CAA0
:1021D0001A6FFA71D645E70FEB3909B35A131FAAE4
:1021E0003A93CF8D6ECAEC2C8EC5831B5AD6D189FB
:1021F000AC024FCB0F257696E05D2CFFA7EAEA9262
:10220000F1725BEE08D8848AA959E31277DAD6CA4C
:102210004E362D7CA413D1E818319902540AD07A95
:1022200074A0AD2C834A6FF1B1501B6469E8842F10
:102230002CC8EB953DA518C74B82FC88E1D37B0EDB
:10224000BE10BA6502859B469A377A774DC2C45351
:1022500030679154F63D39444342132E0929FD500D
:10226000A6DA94CE8697102B5C1C09CD0FFC15DCEA
:10227000543B53E17CA7E1FD47C2AF7EEA34000046
:1022800000000C6FE65C04306C84C751E3B55F342A
:102290009EDD05000000000C1CD4BCFBCD3AAEBC9A
:1022A000529254852CED0FFB00000000F873105D76
:1022B000D81F06E0A15926B4393FC119F9D4BE4F41
:1022C000F433EC3F3FFE8F91D044F21278909E7928
:1022D000A927EE05CB9F5A4B15DE6739181FE73A41
:1022E0000A4198E7DEA728A0D354663379B53A832C
:1022F000375F25407047B8796B62963F48EA9F6E1A
:10230000CB35E16F2DC4C24B9BA74D05790E1CFE4A
:10231000095A9F87227A131B9F994D05DB1573D8A5
:1023200065FE395EA4437B6C79BD73914C9B4C94E4
:102330001887EA68A7449F5C3666FD41145EB18E3B
:10234000EB45DA770EE0EC5EF40DBF41C648F015C0
:10235000D860F74076237B1CE559445030CE064EBA
:10236000C5A670C31817A237ACBF2C6FBC9B3F58D3
:10237000121110390018DB7D0BD22CEE0AAF7694C7
:102380007AC15C21D2619F1D7A9695DFA45181E6C6
:102390001BD57C3644F060FF3AF632EC8FE09AC7EA
:1023A000E3BCADEBA694714B6D000000000000385B
:1023B000974C36A275FFFB3FEB60E131B1BC327741
:1023C0006CBD49934BC207BAF067FD68CAF5A4FF1C
:1023D0002A5EE2BEB569B2A063931BB4BD4612FA91
:1023E000EE885F46DFB2BAE8BA5447EA000018FA4E
:1023F0000891779B1C878B01709EC0052BAAD7AFD5
:1024000030A8018B28A0F59599325F0000000000EC
:102410000008C4EF65453CC36DEFB8349D1C000057
:10242000000000000000046686F2BC9D8797BE0095
:102430000000000008DD58DD530F7DEC930BB95B05
:10244000E30000000000000000087615DFC7682FD9
:10245000A8F84D338FAE0000000000000000088493
:10246000C3E8CB9C718009D71163210000000000F4
:10247000000000040EC6F0509E0AA799000000005C
:1024800000149A5AF9AA5F06DF5C52374B390C7E6A
:1024900018C1ABD636F578BD9F790000000EF23337
:1024A000610EC30B5A24023F42353DA4ADC53050E6
:1024B000000076E7E34508661821EBDD1476F8F1B5
:1024C00055E83B9D8B9392FFA7803438C2AD7CFFCB
:1024D000BD232B0B2C5FEAC09500FB8C376B8A4227
:1024E000913EEFD65143216F803EBDF2B32407A544
:1024F000924A76513172354725E7B9D0F4C2DD52A0
:10250000353A23C416FA2A8D99D0B953C2125C3FCA
:10251000CE8DDBD1C8D159E588FF4911ABAB7BD15A
:10252000F2B43749A0B1FEFE6C08761D0B00000026
:102530009AF4B16DA0F220E417A74D85B38E7ACB43
:102540008730AF119020A819EA2207FAC14CE8FCA5
:10255000A2038F2AC536E4AF669BBA0ADD6590DA1E
:10256000D72762D9193BABF666892DA53070E9AA49
:10257000E2D9C12347FD9A254A5F896297614B9151
:10258000FC341BFC97B27B87F454FCD63648C287D8
:1025900079A3C48F42B13147DDE8D00A714722F3F5
:1025A000F49F287A700CBC5930E0E4132465BD4CCC
:1025B0000E6D9E4D15901972C928B6950E92F97937
:1025C0005C64B9B97BD7DCB4B9B4967F7255AE0000
:1025D000001EB0028E45BDF0A590B7301240B64047
:1025E0009CF16263726DF0BA1AF6F0406A47A2FC81
:1025F0009BD87019000000000000001AF524F64D69
:102600002F64FDF7C3FDA7455D94318FD69F5D21F3
:102610006641D43951AF618C1E9F00000000061145
:10262000E97A8831E126B61C7400000006F5983579
:10263000171AAB193A8CC60000000E7E14D06E44F7
:102640001C666167F18E287230D2BF7D6F00000872
:10265000179962EE7818543AD57F61AC00000000FB
:102660000000000010833E2C924F5A985997FB822D
:1026700097ADC873A26C0D06CF00000000000000EB
:102680000A69DAEB9EF7677FDEE8830B465A3F0064
:10269000000000000002B3607FDCA3FF0000000028
:1026A000000000148ECFA26572CE3E11392D949495
:1026B000478EC78C706B7C498E3CD74C0000000263
:1026C000C877A5FDBA9A000000000000000A1A1B96
:1026D000D94A8303DFE2756E28D9631F000000002A
:1026E0000000021827278F4BE700000000000000C1
:1026F000000000A902C8A1AD308D14000000080040
:1027000002010000030407000000000000000000B8
:10271000000000250028002B0000000000240027F6
:10272000002A000404040404040404020202020255
:102730000203030303030301020408102040800185
:102740000204081020010204081020009730112410
:102750001FBECFEFD8E0DEBFCDBF13E0A0E0B1E0F9
:10276000EEE1F5E702C005900D92A23CB107D9F762
:1027700025E0A2ECB3E001C01D92A53FB207E1F74E
:1027800013E1C7EAD3E104C02197FE010E94733A26
:10279000C63AD107C9F70E9451310C948D3A0C9476
:1027A000000091E09093BD048093DF041092BE047A
:1027B0001092E00408950895089590938104809301
:1027C0008004FC01228121111AC0828580937F043C
:1027D00080EE96E1909388048093870410928A0497
:1027E0001092890480E096E190938404809383049E
:1027F000109286041092850410928204089510921B
:102800007F04E6CF81E480937C0080917A0080642D
:1028100080937A0080917A0086FDFCCF80917800C9
:1028200090917900089590E0FC01E550F94D2491D4
:10283000FC01E95CF84D3491FC01ED5DF84DE4914B
:10284000EE23C9F0222339F0233001F1A8F421301E
:1028500019F1223029F1F0E0EE0FFF1FE15FF84D92
:10286000A591B4918FB7F894EC91611126C0309581
:102870003E233C938FBF08952730A9F02830C9F03C
:10288000243049F7809180008F7D03C080918000C3
:102890008F7780938000DFCF84B58F7784BDDBCFC7
:1028A00084B58F7DFBCF8091B0008F778093B0008F
:1028B000D2CF8091B0008F7DF9CF3E2BDACF3FB7DA
:1028C000F8948091540490915504A0915604B091CD
:1028D000570426B5A89B05C02F3F19F00196A11DEE
:1028E000B11D3FBFBA2FA92F982F8827BC01CD015A
:1028F000620F711D811D911D42E0660F771F881FB9
:10290000991F4A95D1F708958F929F92AF92BF92E7
:10291000CF92DF92EF92FF926B017C010E945F14D5
:102920004B015C01C114D104E104F104B9F00E942F
:102930005F14681979098A099B09683E734081050B
:10294000910580F321E0C21AD108E108F10888EE70
:10295000880E83E0981EA11CB11CE4CFFF90EF907D
:10296000DF90CF90BF90AF909F908F90089580910F
:102970008C0590E0FC01E95CF84D24918D5D984D4B
:10298000FC018491882399F090E0880F991FFC0145
:10299000E75EF84DA591B491FC01E15FF84D85919A
:1029A00094918FB7F894EC91E22BEC938FBF6AE08F
:1029B00070E080E090E00E94841460E080918C05DB
:1029C0000E9413146AE070E080E090E00E9484149A
:1029D00061E080918C050E9413146AE070E080E051
:1029E00090E00C9484142FB7F89460915004709187
:1029F000510480915204909153042FBF089508957B
:102A0000AF92BF92CF92DF92EF92FF920F931F93FC
:102A1000CF93DF936C017B018B01040F151FEB013A
:102A20005E01AE18BF08C017D10759F06991D601F1
:102A3000ED91FC910190F081E02DC6010995892B63
:102A400079F7C501DF91CF911F910F91FF90EF9022
:102A5000DF90CF90BF90AF900895E0918704F09100
:102A600088042091890430918A04A9014170552776
:102A7000309719F44115510579F035952795820F56
:102A8000931F452B41F0DC012D913C91E20FF31F88
:102A90000190F081E02D099581E090E00895842F68
:102AA00080950895E091ED04F091EE040994E09191
:102AB000EF04F091F0040994E091F104F091F20434
:102AC0000994CF93C82FE0914D04F0914E043097B4
:102AD00051F090915A04809158044C2F6091590400
:102AE000890F0995C82F8C2F0E94571581110AC094
:102AF0000E9452150E945C1580E40E9457158C2F8D
:102B00000E945715809158048F5F80935804CF918D
:102B100008950E945C1580E00C9457150F931F9345
:102B2000CF93DF93082F162FD0915C04D80FC0915C
:102B30005B04C60FC770C06B0E9489158C2F0E9462
:102B400057158D2F82958F7080610E9457158D2F9C
:102B50008F700E9457150E94521500935A041093CB
:102B6000590410925804DF91CF911F910F9108954D
:102B70001F93CF93DF93C0E08091D301C817E8F48F
:102B80006C2F80E00E948E158091D20190915A04A2
:102B9000182F191B81F080935A040E945C1580E461
:102BA0000E945715D0E080E00E946115DF5F1D1381
:102BB000FACF0E945215CF5FDFCF60E080E0DF9157
:102BC000CF911F910C948E158091820401C0660FE5
:102BD0008A95EAF790915904960F90935904809141
:102BE000D301482F461B550B9417150621F01CF0F6
:102BF000861B809359046091590480E00C948E15D3
:102C0000AF92BF92CF92DF92EF92FF920F931F93FA
:102C1000CF93DF93A0918004B091810412961C9110
:102C20001297C62FD0E011110DC014962C91149755
:102C3000AE01421B51091896ED91FC911997E40FD2
:102C4000F51F14911396BC9000917F04E12EF12C96
:102C500040915A042091D20130E02E193F094217C9
:102C6000130621F01CF06B2D0E94E41580915A048C
:102C70008E0D9F2D911D800F911D2091D20128173F
:102C800019060CF400E0A0918004B0918104149620
:102C90008C911497C81BD109A9F012968C911297A8
:102CA00013969C911397492F50E0882311F1899F27
:102CB000C00111249E01289FE001299FD00D389F5B
:102CC000D00D1124AB2C0E945C1580E40E94571596
:102CD000CE01282F2C1B211708F441C0CE0DDF1D7B
:102CE000D12C0D1509F44DC080E00E946115D394DC
:102CF000F8CFBE01F4E076956795FA95E1F730E0FC
:102D000020E090E080E06217730781F06901CC0C4D
:102D1000DD1C1696ED91FC911797EC0DFD1DC590ED
:102D2000D4908C0D9D1D2F5F3F4FEDCF9E01207FD6
:102D30002C173D0760F41896ED91FC911997E20F5E
:102D4000F31FE4918E0F911D2F5F3F4FF1CF849FB2
:102D5000E001859FD00D949FD00D1124B3CF6C015D
:102D60004FEFC41AD40AE0918004F09181040190DD
:102D7000F081E02DE80FF91F84910E946115C601D2
:102D8000A8CF0E9452156091590451E06F5F809165
:102D90005A045A1528F06B1980915A04810F800F3C
:102DA0000E948E15AA94A1108ECFDF91CF911F9112
:102DB0000F91FF90EF90DF90CF90BF90AF9008956C
:102DC0006D3039F1E0918004F09181046A3019F49A
:102DD00063810C94E41524816217D8F025812617AD
:102DE000C0F02091850430918604A901559547953E
:102DF000840F951FE0918304F091840420FF08C0A4
:102E0000DC012D913C91E20FF31F0190F081E02D48
:102E10000994089520912A04260F3327331F213265
:102E20003105ECF42091B704FC0190E080E02430FF
:102E300069F082E00895A0912A042191AC01465FD7
:102E40005B4FA40FB52FB11D2C930196861798F3F5
:102E500080912A04680F60932A0480E0089581E03D
:102E600008951092B70481E08093B6041092910403
:102E700061E082E10E94131461E083E10E94131477
:102E8000E9EBF0E080818E7F808380818D7F80837D
:102E900088E48093B80085E48093BC000895109284
:102EA000900410928F041092BE041092E0040E94CD
:102EB00031178BED93E190938E0480938D048CED0C
:102EC00093E190938C0480938B040895CF93DF93C8
:102ED00091E0909309048823B9F0C091B800D09193
:102EE000BA008091BC008A7B8093BC0060E082E1E4
:102EF0000E94131460E083E10E9413140E943117B2
:102F0000D093BA00C093B800DF91CF910895CF92CB
:102F1000DF92EF92FF920F931F93CF93DF93D091A5
:102F2000E00481E0D13208F09CC0C091DF040E942F
:102F30005F146B017C018091B70481116CC082E049
:102F40008093B70481E08093B6048FEF8093B5043B
:102F50001092B404D093B304AFEBB4E0E3E9F4E02F
:102F600080E0D8138DC01092920480919204CC0F0F
:102F7000C82BC093920480919104813009F084C0E1
:102F8000109291040E945F146B017C018091920465
:102F90008093BB008091B9049091BA04A091BB04C6
:102FA000B091BC04892B8A2B8B2BA1F00E945F145B
:102FB0000091B9041091BA042091BB043091BC0473
:102FC0006C197D098E099F0906171707280739070D
:102FD00008F442C08091BC0083FDD8CF85EC80937B
:102FE000BC000E945F146B017C018091B7048230A9
:102FF00009F44CC08091B5048F3F09F469C08091F9
:10300000B504803209F466C08091B504803309F4B8
:1030100063C084E026C08091B9049091BA04A09165
:10302000BB04B091BC04892B8A2B8B2B09F483CF72
:103030000E945F140091B9041091BA042091BB045E
:103040003091BC046C197D098E099F09061717077A
:103050002807390708F06FCF8091B8040E946617DF
:1030600085E01092BE041092E0041092BD04DF913E
:10307000CF911F910F91FF90EF90DF90CF90089527
:103080009D9191938F5F6DCF85EEA9CF8091B9040B
:103090009091BA04A091BB04B091BC04892B8A2BF7
:1030A0008B2B09F4A2CF0E945F140091B9041091F8
:1030B000BA042091BB043091BC046C197D098E09BF
:1030C0009F09061717072807390708F08ECFC4CFC6
:1030D00080E0C7CF82E0C5CF83E0C3CF0C948717D1
:1030E0000895E091900480918F04E81730F4F0E0A7
:1030F000E15AFB4F808190E008958FEF9FEF089594
:103100009091900480918F042FEF3FEF981748F42F
:10311000E92FF0E0E15AFB4F208130E09F5F909370
:103120009004C901089580918F0490919004891BA7
:10313000990B0895CF92DF92EF92FF920F931F9316
:10314000CF93DF937C01CB018A012091BD04222320
:1031500089F0EB016B01C40ED51ECC15DD0569F0BD
:103160006991D701ED91FC910190F081E02DC701AB
:103170000995F3CF642F0E940A17C801DF91CF9100
:103180001F910F91FF90EF90DF90CF900895CF9314
:10319000DF931F92CDB7DEB769832091BD04222350
:1031A000F9F02091E004203258F021E030E0FC01F9
:1031B0003383228390E080E00F90DF91CF910895D8
:1031C0008091BE04E82FF0E0E154FB4F9981908399
:1031D0008F5F8093BE048093E00481E090E0ECCFA9
:1031E00061E0CE0101960E940A17F7CF682F81EEA9
:1031F00094E00E94C71821E0892B09F420E0822F77
:103200000895682F81EE94E00C94C718CF92DF9256
:10321000FF920F931F93CF93DF938C01EB010E94DA
:10322000F314607F7370F801A081B1819D012F704C
:103230003327AD01407F5370FB2EF694F694F7E0F0
:10324000FF15F8F089B190E00F2C02C09595879595
:103250000A94E2F781706417750708F47C5F6B01CC
:10326000C41AD50A2730310508F5F901E65CF64E97
:103270000C94733A5319581999195D1980198919C1
:103280009219EF2DF0E08DE08F1548F083B190E0BA
:10329000389702C095958795EA95E2F7DBCF86B11E
:1032A00090E03E97F6CF882309F44BC080E00DC034
:1032B0008823E1F130E020E0F9CF811146C090E4AD
:1032C000C91691E0D90608F044C0AA27BC7FA22BFA
:1032D000B32B407F53704A2B5B2BF8015183408303
:1032E000882309F440C0209709F441C06F2DFE01E6
:1032F000DF91CF911F910F91FF90DF90CF900994B4
:1033000081112CC0E0E3CE16D104F8F2AB0187E0C6
:10331000DCCF24E030E08823C1F2AB0122E030E0D2
:103320008BE0D3CF22E030E08111CFCF23E030E03B
:10333000CCCF8823B1F0F0E4CF16D10408F0BACF97
:10334000B5CFAB0121E030E0C0CFAB0126E030E0EB
:10335000ADCFAB0124E030E083E0B7CF25E030E033
:10336000A5CFAB01B2CF2330310508F088E0DF9163
:10337000CF911F910F91FF90DF90CF900895E09132
:103380000704F09108043097A1F01082E091050441
:10339000F0910604309709F00995109201041092FB
:1033A0000204109203041092040410920804109274
:1033B00007040895833009F481E00895FC018081B9
:1033C000280F261714F440830895421714F0208321
:1033D000089560830895282F41E060E080EC91E03B
:1033E0000C94DE19282F41E060E087EB91E00C940B
:1033F000DE19282F41E060E08CE991E00E94DE199F
:10340000F894E1E6F0E080E8808380919C0180837D
:1034100078940895282F41E060E081E891E00C94D1
:10342000DE19CF93282F4DE765E088E791E00E94F1
:10343000DE19C0917801CC0F0E94891581E80E94A5
:1034400057158C2F0E945715CF910C9452150C9440
:103450002D158091E703811103C086B1809581709D
:1034600008950E94F3146093ED057093EE05809328
:10347000EF059093F0051092E9031092E803089588
:1034800089B199B1E091D805EF70869586958270E3
:1034900092FB992790F9892B94E0E99FF001112480
:1034A000E450FE4FE80FF11D87FDFA95808180936F
:1034B000D805807359F0803151F08FEF9FEF9093D2
:1034C000FB038093FA0381E08093E703089581E092
:1034D00090E0F5CF80913C01882329F090913C0148
:1034E00081E0943008F080E008950E946A1A81110A
:1034F00003C086E090E008958BE090E008950E947C
:103500006A1A8823C9F080911801E0911801EE0F22
:10351000FF0BEB59FD4F87301CF08081918108959E
:103520004081518128EE33E0429FC001439F900DBE
:10353000529F900D1124089580911801873014F046
:1035400010921801E0911801EE0FFF0BEB59FD4F9F
:10355000E4CF8A30910568F08436910568F0883EA2
:1035600023E0920760F08031974260F085E090E0C0
:10357000089581E090E0089582E090E0089583E06E
:1035800090E0089584E090E00895CF92DF92EF926A
:103590000F93CF93DF93EC01EFEFE40F0E2E000CAF
:1035A000FF0B8AE0C82ED12CE7FD0BC0CB01B60182
:1035B0000E940A3ADE01AE0FBF1F805D8C933197E7
:1035C000F3CFFE01E40FF11D1082222389F0822F38
:1035D00090E0AF014C1B5D0B4817590724F0308178
:1035E00031833197F6CF8C0F9D1FFC010083422F52
:1035F000415080E050E0E82F082E000CFF0BE4174C
:10360000F50744F4EC0FFD1F9081903319F48F5FA0
:10361000E082F1CFDF91CF910F91EF90DF90CF90CB
:103620000895009769F02091010130910201281757
:10363000390731F090930201809301010C94DD135E
:1036400008958CE30E94D11381E008950E944F17E2
:103650000E94211B0E946E18882339F06AE070E0F6
:1036600080E090E00E948414F3CF0895089590E0E4
:1036700080E008958F929F92AF92BF92CF92DF9297
:10368000EF92FF921F93CF93DF93D82F162F0E94B4
:103690005F146B017C018091B704811166C0C12F5A
:1036A00081E08093B7048093B6049FEF9093B504B4
:1036B0001092B404910F9093B3048093920480917C
:1036C0009204DD0FD82BD093920480919104813025
:1036D00009F082C0109291040E945F146B017C017A
:1036E000809192048093BB008091B9049091BA04B8
:1036F000A091BB04B091BC04892B8A2B8B2BA1F029
:103700000E945F148090B9049090BA04A090BB040A
:10371000B090BC046C197D098E099F098616970626
:10372000A806B90608F442C08091BC0083FDD8CF3A
:1037300085EC8093BC000E945F146B017C0180913A
:10374000B704813009F44AC08091B404811710F4A1
:10375000C091B404A3E9B4E0EFE5F4E080E08C1795
:1037600051F19D9191938F5FFACF8091B90490911F
:10377000BA04A091BB04B091BC04892B8A2B8B2B7B
:1037800009F489CF0E945F148090B9049090BA0424
:10379000A090BB04B090BC046C197D098E099F09F0
:1037A00086169706A806B90608F075CF8091B8046A
:1037B0000E946617C0E010929004C0938F048C2F73
:1037C000DF91CF911F91FF90EF90DF90CF90BF904E
:1037D000AF909F908F90089585EEABCF8091B90404
:1037E0009091BA04A091BB04B091BC04892B8A2BA0
:1037F0008B2B09F4A4CF0E945F148090B9049090A1
:10380000BA04A090BB04B090BC046C197D098E0969
:103810009F0986169706A806B90608F090CFC6CF6E
:10382000CF93DF93CBEAD4E0CE010197F1F761E0CB
:1038300070E080918105909182050E943A1B81EE93
:1038400094E00E94801887FFEFCFDF91CF91089519
:103850000F931F93CF93DF93182F092FEB010E9433
:10386000101C809181050E94D11382E190E00E949A
:10387000011990E080E00E940119602F81EE94E030
:103880000E94C718612F81EE94E00E94C7186D2F27
:1038900081EE94E00E94C7186C2F81EE94E00E94A4
:1038A000C7180E94871783E998E00197F1F7DF9125
:1038B000CF911F910F910895CF93C82F682F70E07B
:1038C00080E090E40E94281CC093D405CF91089515
:1038D000282F41E060E086E691E00E94DE198091A9
:1038E0003C01843059F48091660162E0811101C08D
:1038F00061E070E080E091E10C94281C0895282F8D
:103900004AE56CE08FE691E00E94DE1980913C016F
:10391000843099F080916F0194EF980F9F3468F490
:103920008093970524E531E0829FB001839F700D5D
:10393000112483E091E30C94281C0895282F40E281
:1039400060E08BE491E00E94DE1980913C018430BC
:1039500039F060914B0170E082E093E30C94281CF5
:1039600008950E94101C809181050E94D11382E16C
:1039700090E00E94011990E080E00E94011961E04E
:1039800081EE94E00E94C71861E081EE94E00E940D
:10399000C7186091D10581EE94E00E94C71860912C
:1039A000D00581EE94E00E94C7180E94871783E932
:1039B00098E00197F1F70895282F41E060E08AE848
:1039C00091E00E94DE190E946A1A882351F08091CA
:1039D000D10590918A0190FB85F98093D1050C94D3
:1039E000B11C0895909193018091D005992329F0FD
:1039F00020913C0191502330A1F4E09105012E2F3C
:103A0000EE0F330BF901EE0FFF1FE20FF31FEB5622
:103A1000FD4F2081222321F0245091E0223008F430
:103A200090E09295907F8F70892B8093D0050C94B5
:103A3000B11C282F42E060E083E991E00E94DE198A
:103A40000E946A1A81110C94F21C0895CF93DF939F
:103A5000D82FC92F0E94101CD093A005C093A10598
:103A6000C093A305D093A4059091D605992361F046
:103A70008091A2059295990F990F907C8370892B64
:103A800081608D7F8093A205809181050E94D11372
:103A900060918D0581EE94E00E94C7186091A205A7
:103AA00081EE94E00E94C7186091A30581EE94E036
:103AB0000E94C7186091A40581EE94E00E94C71887
:103AC0006091A50581EE94E00E94C71880918D0554
:103AD000803431F46091A60581EE94E00E94C7180D
:103AE0000E9487170E94101CD0939205C0939305E3
:103AF000609183057091840590E080E0DF91CF9123
:103B00000C9484148091D70587FD07C061E00E9462
:103B100013148BEA94E00197F1F70E94101C809136
:103B200081050E94D11381E190E00E9401190E9459
:103B300087178BE097E20197F1F70895CF93909163
:103B40008D05903459F5873048F5C82FCF700E9405
:103B5000101C809181050E94D11382E190E00E94A7
:103B6000011990E080E00E94011961E381EE94E088
:103B70000E94C71862E081EE94E00E94C71861E0DD
:103B800081EE94E00E94C7186C2F81EE94E00E94B1
:103B9000C7180E948717CF910C94101CCF910895DD
:103BA0001F93CF93DF930E94101C809181050E9488
:103BB000D11381E090E00E9401196091D20581EE5D
:103BC00094E00E94C7186091D30581EE94E00E94B2
:103BD000C7180E9487170E94101C6091850570917C
:103BE000860590E080E00E9484148091D70587FDCF
:103BF00007C060E00E9413148BEA94E00197F1F78C
:103C00008091980581111EC0C0919B05D0919C05A3
:103C1000BE0181E092E00E94281CD0939C05C093D5
:103C20009B0510919F05C0919D05D0919E05BE01F9
:103C300082E092E00E94281CD0939E05C0939D05CF
:103C400010939F05DF91CF911F9108951F93CF93FC
:103C5000DF93C091420181E0C11103C080E0C0E068
:103C600003C0C230E0F3C15090918D05D8E290328C
:103C700021F0D8E4903509F4D8E510E080FB10F984
:103C80000E94101C809181050E94D1136D2F81EE3E
:103C900094E00E94C718612F81EE94E00E94C7183B
:103CA0006C2F81EE94E00E94C7180E948717DF9165
:103CB000CF911F910C94101C282F45E260E082E404
:103CC00091E00E94DE190C94261ECF93DF93809121
:103CD0008D058032A1F1C091AE0186EFC802E001EE
:103CE00011248091EB039091EC03C81BD90B0E9427
:103CF000101C809181050E94D11382E190E00E9406
:103D0000011990E080E00E94011961E081EE94E0E9
:103D10000E94C71860E081EE94E00E94C7186D2FE2
:103D200081EE94E00E94C7186C2F81EE94E00E940F
:103D3000C7180E94871783E998E00197F1F7DF9190
:103D4000CF910895FF920F931F93CF93DF93182F76
:103D500080918D05803251F0C8E0D0E002E48034DB
:103D600041F0C6E0D0E002E5803519F0C8E0D0E0CF
:103D700002E20E94101C110F1270809181050E94B6
:103D8000D113602F81EE94E00E94C718612F81EE5D
:103D900094E00E94C7180E9487170E94101CBE0161
:103DA00080918105909182050E943A1BF12C0F2D84
:103DB00010E00C171D0754F481EE94E00E94801867
:103DC000F801E155FA4F8083F394F1CF8091AF056C
:103DD00086FDE3CFDF91CF911F910F91FF900C945F
:103DE000101C81E00E94A21E8091B2059091B10545
:103DF000E2E9F5E08083918308958F929F92AF92DC
:103E0000BF92CF92DF92EF92FF920F931F93CF93C7
:103E1000DF93CDB7DEB728970FB6F894DEBF0FBE9D
:103E2000CDBF88E08093B8000E94821D0E94101CC4
:103E3000809181050E94D11381E090E00E940119D8
:103E40008FE190E00E94011985E090E00E94011945
:103E50000E9487177E0129E0E20EF11C0E94101CCF
:103E600068E070E080918105909182050E943A1B84
:103E70008E010F5F1F4F81EE94E00E948018F801C1
:103E800081938F01EE16FF06B1F7898186FDE6CF9B
:103E90008BE097E20197F1F70E94101C8091810559
:103EA0000E94D11381E090E00E94011981E390E02B
:103EB0000E94011985E090E00E9401190E94871775
:103EC000609185057091860590E080E00E948414E1
:103ED00062E370E080E090E00E948414D12CC12C59
:103EE00010E000E05BEAA52E54E0B52E80E598E0F6
:103EF000FC0125913491C216D30609F471C00296D3
:103F0000F8E08E3B9F07A1F746E1F42E80918105F2
:103F10000E94D1136F2D81EE94E00E94C718F12CFE
:103F2000E12CC8018254974F4C01F401EE0DFF1DA6
:103F3000649181EE94E00E94C7189FEFE91AF90A94
:103F4000E7E0EE16F10489F70E948717C501019793
:103F5000F1F7FFEFCF1ADF0A095F1F4F07332EE19A
:103F6000120709F0C3CF83EE93E00197F1F7809138
:103F70008D058032D1F0E09105018E2FEE0F990B67
:103F8000FC01EE0FFF1FE80FF91FEB56FD4F80817C
:103F90008F7080618093D0058091D1058078806199
:103FA00080688093D1050E94B11C88E48093B8009A
:103FB00081E08093EA031092180128960FB6F894D6
:103FC000DEBF0FBECDBFDF91CF911F910F91FF904C
:103FD000EF90DF90CF90BF90AF909F908F9008951B
:103FE00035E1F32E93CFCF93DF938091920590919B
:103FF000930520915D0430915E0482179307C9F008
:1040000090935E0480935D04E5EFF4E081E4DF01CA
:104010001D928A95E9F7E6E3F5E081E2DF011D9262
:104020008A95E9F7E7E5F5E089E0DF011D928A95D9
:10403000E9F70E94101CC0E0CE7FCD7FCB7F80913E
:1040400081050E94D11384E290E00E9401196C2F37
:1040500081EE94E00E94C7180E9487170E94101CEE
:104060006DE070E080918105909182050E943A1B7D
:10407000C0ECD5E081EE94E00E9480188993B5E011
:10408000CD3CDB07B9F78091C00586FDE7CF83E91A
:1040900098E00197F1F7DF91CF910895CF93C82F62
:1040A0000E94101C8C2F8370282F2295207FC82FF0
:1040B000C295CC0FCC0FC07C982F990F990FC22BB3
:1040C000C92BC82B809181050E94D11382E190E019
:1040D0000E94011990E080E00E94011965E181EEE3
:1040E00094E00E94C71862E081EE94E00E94C71835
:1040F0006C2F81EE94E00E94C71861E081EE94E09D
:104100000E94C7180E94871783E998E00197F1F78A
:10411000E5EFF4E081E4DF011D928A95E9F7E6E33B
:10412000F5E081E2DF011D928A95E9F7E7E5F5E028
:1041300089E0DF011D928A95E9F710927E051092C1
:104140007D0510928B0510927C0510927B051092D4
:104150007A0510927905CF910895282F43E060E009
:1041600085EA91E00E94DE1980913C01843021F4BF
:104170008091A5010C944E200895282F4CE364EC07
:104180008EEA91E00E94DE190E946A1A882331F0BB
:104190008091AE010E944E200C94651E08958F926E
:1041A0009F92AF92BF920F931F93CF93DF93CDB7A0
:1041B000DEB7A1970FB6F894DEBF0FBECDBF19A230
:1041C000423008F44AE08E010F5D1F4F842E912C7F
:1041D000B12CA12CA50194010E94323AE62FB9011D
:1041E000CA01EA3044F5E05DD801EE938D01232B3E
:1041F000242B252B79F790E080E0109769F0FD01E2
:1042000001900020E9F73197AF014A1B5B0BBD011C
:1042100081EF95E00E940015A1960FB6F894DEBFDD
:104220000FBECDBFDF91CF911F910F91BF90AF9087
:104230009F908F900895E95CD7CF009769F0FC01BB
:1042400001900020E9F73197AF01481B590BBC01E1
:1042500081EF95E00C94001590E080E00895CF92F6
:10426000DF92EF92FF920F93CF93DF93EC017B01EC
:104270006A01C9010E94111B002361F08FE495E1DE
:1042800090934E0480934D04F7FE12C0CE010E941D
:104290001D2119C0F7FC02C0D7FE0CC0CE01DF9172
:1042A000CF910F91FF90EF90DF90CF900C941D2154
:1042B000D7FCECCF6C2D8E2D0E948E15CE010E9466
:1042C0001D21002321F010924E0410924D04DF9125
:1042D000CF910F91FF90EF90DF90CF9008950F93C3
:1042E0000E946A1A882301F1E09105018E2FEE0FDA
:1042F000990BFC01EE0FFF1FE80FF91FEB56FD4F66
:104300008181928120913C01233011F480ED92E073
:104310000091F10327EA32E050E040E06DE270E006
:104320000E942F210F91089580913C0181110FC0AF
:10433000E09104018E2FEE0F990BFC01EE0FFF1F91
:10434000E80FF91FE058FD4F81819281E1CFE091A4
:10435000E603EE0FFF0BEB5CFD4F80819181D8CF20
:10436000DF92EF92FF920F931F93CF93DF93CDB71E
:10437000DEB761970FB6F894DEBF0FBECDBF0E94C7
:10438000F3140091E1031091E2032091E3033091D3
:10439000E403601B710B820B930B6436710581057E
:1043A000910508F46BC080918D0528E0E22EF12C78
:1043B00013E2803251F036E0E32EF12C13E4803525
:1043C00021F498E0E92EF12C13E50E94101C809155
:1043D00081050E94D113612F81EE94E00E94C718DD
:1043E00060E081EE94E00E94C7180E9487170E9447
:1043F000101CB70180918105909182050E943A1BA3
:10440000D12C0D2D10E00E151F0554F481EE94E013
:104410000E948018F801E955FA4F8083D394F1CFB8
:104420002091AB05213408F020E430E03595279544
:1044300035952795FE01319650E040E0CF016CE7BD
:10444000421753070CF060E261934F5F5F4F4031BA
:104450005105A9F7198A01E027EA32E046E050E069
:1044600070E060E00E942F210E94F3146093E1034A
:104470007093E2038093E3039093E40361960FB695
:10448000F894DEBF0FBECDBFDF91CF911F910F918A
:10449000FF90EF90DF900895EF920F93CF93DF930B
:1044A00000D000D01F92CDB7DEB78091F703811105
:1044B00066C08091EE03811162C080913C0184301E
:1044C00011F5E09103010E2E000CFF0BE358FD4F98
:1044D0006081643649F480E289838A8381E38B8337
:1044E0008DE48C831D8233C02AE06202B001112466
:1044F00080E2E82E00E020E043E0CE0101960E9439
:10450000C51A8BE6EECFE0911801EE0FFF0BEB59C9
:10451000FD4F80819181883E9340E9F20E946A1AA2
:104520008823B9F18091180187309CF1E09118013E
:10453000EE0FFF0BEB59FD4F6081718190E2E92E88
:1045400000E020E044E0CE0101960E94C51A0091EF
:10455000F20327EA32E046E050E06EE170E085EDDC
:1045600092E00E942F210091F20327EA32E046E018
:1045700050E06AE370E0CE0101960E942F210F9077
:104580000F900F900F900F90DF91CF910F91EF90C0
:104590000895E0911801EE0FFF0BEB59FD4F60817C
:1045A0007181A6CFEF92FF920F931F93CF93DF936A
:1045B0008091D90381110DC00E94F3146093D5033B
:1045C0007093D6038093D7039093D80381E08093B0
:1045D000D90380913C01843009F05BC18091EE03E6
:1045E000882309F456C18091F603811152C10E94BB
:1045F000F3140091D5031091D6032091D703309185
:10460000D803601B710B820B930B6D3271408105D7
:10461000910510F01092D1038091ED034091D303E6
:104620005091D4032091F8033091F90342175307B6
:10463000E1F481111CC08091F8039091F9039093EB
:10464000D4038093D303C091D103CC2369F180912B
:10465000ED038111AAC0CC2309F4A7C0DF91CF914B
:104660001F910F91FF90EF9008958823C1F08091E2
:10467000D0038F5F833080F48093D0031092D203F5
:1046800000E027EA32E046E050E070E060E087E0DA
:1046900091E00E942F21CFCF1092D003EFCF109244
:1046A000D0031092D103EACF80918D05803211F4AE
:1046B0000E94F31F8091C10580FFC9CF8091C20580
:1046C00080FFC5CF8091C305823008F4C0CF8091B0
:1046D000C60582958F7009F07CC020918B05809172
:1046E000C70584FB992790F9291749F090938B050A
:1046F000E7E5F5E099E0DF011D929A95E9F783700F
:1047000090E090937E0580937D05880F991FFC01B2
:10471000E95AFA4F2091CB0521832091CA052083C5
:1047200010925F0587E595E09093CB038093CA03D1
:104730008091C60582958F70B0E0A0E08230B9F418
:104740008091C7058F7090E090937C0580937B05E6
:10475000880F991FFC01EA5CFA4F2091CB05218359
:104760002091CA05208310925605A6E3B5E0B093C8
:10477000CD03A093CC038091C10580FD2DC0F0E056
:10478000E0E0F093CF03E093CE0351961C92118AA0
:1047900081E08093D1030E94F3146093D50370935A
:1047A000D6038093D7039093D803E091D003F0E031
:1047B000EE0FFF1FE653FC4F80819181D0E0ED2E7C
:1047C000F12CFC01EE0DFF1D2081222351F1DF5F52
:1047D000F6CF90E080E0A8CF8091C60582958F70DB
:1047E000823069F6E091C705EF70F0E0F0937A054A
:1047F000E0937905EE0FFF1FEE0FFF1FEB50FB4F0D
:104800008091C80580838091C90581838091CA0504
:1048100082838091CB05838310923405E5EFF4E029
:10482000B0CFD11105C02091ED03222309F416CF9A
:1048300000E027EA32E046E050E070E060E00E94ED
:104840002F21DD23F1F02091D203022E000C330B37
:10485000E216F306CCF42E193F0980E190E08E19A0
:104860009F09281739070CF4C901C82F10E2F12C51
:10487000FC1651F0612F81EF95E00E942D15F39405
:10488000F7CFC3E01EE2F3CFD093D2031092ED0333
:10489000E5CE1092D4031092D3031092D20310925B
:1048A000D1031092D003DACE4F925F926F927F9233
:1048B000AF92BF92CF92DF92EF920F931F93CF935D
:1048C000DF93CDB7DEB7AC970FB6F894DEBF0FBE5F
:1048D000CDBF9091E503992309F4C2C0B82E88E2B8
:1048E000E4EDF1E0DE01119601900D928A95E1F779
:1048F0000E9402146C010091C8031091C90397FD36
:1049000068010E94F3144090C4035090C503609066
:10491000C6037090C7036419750986099709613148
:1049200077428105910518F4BB2009F488C01CA6C4
:1049300064E6033882E0180708F045C0093E91E0BC
:10494000190708F4A6C0FE01319690E080E0AC01A2
:104950000196248135810217130708F495C0608100
:1049600071816017710708F48FC0621B730B880F89
:10497000991F880F991FE1E0F0E0EC0FFD1FE80F91
:10498000F91FA280B380FA01EE0FFF1FEE0FFF1F89
:1049900081E090E08C0F9D1FE80FF91F4281538149
:1049A0004A195B09021B130B409FC001419F900DE8
:1049B000509F900D11249B0136952795820F931FD0
:1049C0000E940A3A6A0DA62EB12CC5010E94A91AAE
:1049D00012E003970CF013E090E2E92E00E020E0F3
:1049E000412FB501CE0189960E94C51A123011F4EB
:1049F00085E28BA78091F603811113C08091F703A4
:104A000081110FC08091EE0381110BC000E027EAF5
:104A100032E046E050E066E670E0CE0189960E9402
:104A20002F210E94F3146093C4037093C5038093F5
:104A3000C6039093C703D092C903C092C803809164
:104A4000C8039091C903C80ED91ED7FE03C09FEFBB
:104A5000C91AD90AD594C794D092C903C092C80381
:104A6000AC960FB6F894DEBF0FBECDBFDF91CF91ED
:104A70001F910F91EF90DF90CF90BF90AF907F90FC
:104A80006F905F904F90089534968930910509F0AA
:104A90005ECF60E098CFEF920F93CF93DF9300D07B
:104AA0001F92CDB7DEB78091F60381111CC08091B3
:104AB000EF03811120C06091D40570E080E2E82E00
:104AC00000E020E042E0CE0101960E94C51A00916C
:104AD000F30327EA32E050E040E06CE670E0CE01FC
:104AE00001960E942F210F900F900F90DF91CF9190
:104AF0000F91EF90089580E289838DE48A831B8271
:104B0000E6CF282F8091EF03882331F00E945C1CB0
:104B10001092EF030C944B259091D405213051F461
:104B20009F3318F49F5F9093D4058091D4050E9421
:104B30005C1CF0CF9923C9F39150F5CFCF93DF934D
:104B4000C82FD62F8091EF03882349F0C3FD07C0FB
:104B5000C13011F4663019F481E00E948125809102
:104B6000EF0381110CC08C2F8370833041F4CB3064
:104B700031F08FEFD63009F481E00E9481258C2F2F
:104B8000DF91CF9108950F938091F703811127C092
:104B90008091EE03811123C00091F003002331F0D6
:104BA00080913C0101E0843009F400E08091F80339
:104BB0009091F903885596468830974090F0E0919F
:104BC0003A01EE0FFF0BE35DFD4F8081918127EAF3
:104BD00032E046E050E070E060E00E942F210F914B
:104BE00008958AED92E0F3CF0F930091F003002334
:104BF00031F080913C0101E0843009F000E0E09167
:104C00003C01F0E0EE0FFF1FED5DFD4F27EA32E0C3
:104C100050E040E070E060E0808191810E942F21AF
:104C200083ED92E00E941D210E946A1A8823A1F060
:104C300080915D01813081F4209101013091020168
:104C400001E04FEF5FEF6FEF7FEF8DED92E00E949D
:104C50002F210F910C94C32583ED92E00E941D211A
:104C6000F8CFEF92FF921F93CF93DF93EC017B017C
:104C70008881D0930804C09307047093060460935E
:104C8000050411E01827811122C01092F30310923D
:104C9000F2031092F1031092F0030E94F314609358
:104CA00001047093020480930304909304040E940F
:104CB0004B250E944C220E946F210E94F4251883EC
:104CC000F701DF91CF911F91FF90EF90099410921F
:104CD0000104109202041092030410920404EFCF16
:104CE0000F9301E027EA32E050E040E070E060E03E
:104CF0008FED92E00E942F218FE495E190934E0476
:104D000080934D046091CD0170E090E080E04AE036
:104D10000E94CF2085EF92E00E941D214AE063E0CF
:104D200070E080E090E00E94CF2010924E0410923C
:104D30004D040F9108958F929F92AF92BF92CF92A0
:104D4000DF92EF92FF920F931F93CF93DF9300D0E8
:104D500000D01F92CDB7DEB79091F603992309F4E6
:104D600066C0C090CD010C2C000CDD0821E0C21AF9
:104D7000D1089C2D990F990F4C2D491B440F480FBA
:104D8000433008F466C04358440F9CE3F82EA82E25
:104D9000B12CC42ED12C892E912C6623E9F0809160
:104DA000F403082E000C990B00E08A159B0521F4F2
:104DB0000091F50381E0082729E0F29EC00111244B
:104DC00027EA32E0A6014E5F5F4FB4016B5F7F4F71
:104DD000835C9E4F0E942F2189E08A9DF0018B9D6C
:104DE000F00D1124E35CFE4F15818681813009F4BA
:104DF0004AC090F1823009F468C0833009F45AC087
:104E00008091F403082E000C990B0091F5038A158C
:104E10009B0509F000E0A6014E5F5F4FB4016D5D98
:104E20007F4F27EA32E0CE0101960E942F210F909A
:104E30000F900F900F900F90DF91CF911F910F91D6
:104E4000FF90EF90DF90CF90BF90AF909F908F90AA
:104E50000895440F90E09ACF111108C081E489832E
:104E600085E58A8384E58B831C82CACF612F110F6D
:104E7000770B90E2E92E00E020E043E0CE010196BE
:104E80000E94C51ABDCF612F012E000C770B77FF52
:104E900003C071956195710980E2E82E00E020E081
:104EA00043E0CE0101960E94C51A17FFA9CF8DE2FB
:104EB0008983A6CF112391F2113009F04BC08FE402
:104EC00089838EE68A8380E2CECF84E0F8120CC01C
:104ED000111106C085E3898380E38A8385E7C3CF08
:104EE00087E3898385E3F9CF97E0F91208C08BE661
:104EF00011118DE4898388E48A838AE7B4CF28E09E
:104F0000F2120CC0111104C082E5898383E525C02B
:104F100083E589838EE48A8382E5A5CF8FE0F8124A
:104F200008C08CE4111185E5898383E58A8382E4D6
:104F30009ACF9AE0F9120CC0111104C081E3898361
:104F400080E30BC085E3898380E38A8385E28BCF8E
:104F50001111B5CF8FE4898386E68A8384CF1F93AE
:104F6000CF93DF93D0E0C0E016E08091CD01082E12
:104F7000000C990B0197189F9001199F300D112477
:104F80002C0F3D1F2031310564F4982F990F890FA4
:104F9000880F61E08C0F0E949B262196C630D105B8
:104FA00021F7DF91CF911F9108950F9300E027EA39
:104FB00032E046E050E070E060E087E091E00E947F
:104FC0002F210E94F4250E944C2281E00F910C9425
:104FD00054248091F703811104C08091EE0388234B
:104FE00031F01092F7031092EE030C94D527089538
:104FF0004F925F926F927F929F92AF92BF92CF92A9
:10500000DF92EF92FF920F931F93CF93DF93CDB771
:10501000DEB72F970FB6F894DEBF0FBECDBF9091CD
:10502000F6039111B7C0982E0E946A1A73E0F72E0A
:10503000811102C06CE0F62E8BE68C8788E48D87A8
:105040008AE78E871F868EE2888780E389878A8732
:105050001B8680913A01833081F46091F80370914E
:10506000F9035FE2E52E0EE223E045E0CE01019672
:105070000E94C51A8DE48C8724C0823011F40E94EE
:10508000C3250E946A1A6091F8037091F903811197
:1050900097C01091810170903A0182E0781203C0AC
:1050A00022E0113009F020E04FE2E42E0EE245E06C
:1050B000CE0101960E94C51A82E0781202C011301A
:1050C000C9F20E946A1A882309F4B1C0C5010E947E
:1050D000A91A182F992009F4AFC063E080E00E945C
:1050E0008E1500E028E132E043E050E070E060E03F
:1050F0008DEE92E00E942F216F2D70E000E028E1FC
:1051000032E043E050E0CE0101960E942F210E9440
:105110006A1A882351F1C6010E94A91AAC01CE0176
:105120004130510509F49FC0099620E2E22E00E0CB
:1051300020E0B6010E94C51A1B8680910101909162
:1051400002010E94111BCE0108960E941D21809130
:10515000C303181750F480910101909102010E943D
:10516000111B85EF92E00E941D218091B7018130D3
:1051700079F40E946A1A811178C000E027EA32E0CF
:1051800044E050E066E670E0CE010C960E942F21CC
:105190001093C3032F960FB6F894DEBF0FBECDBF9A
:1051A000DF91CF911F910F91FF90EF90DF90CF9003
:1051B000BF90AF909F907F906F905F904F900895B9
:1051C0009B01A8EEB3E00E94793A4090EB03509027
:1051D000EC03052C000C66087708640D751D861D10
:1051E000971D28EE33E040E050E00E94543A290138
:1051F000520197FF07C090958095709561957F4FFC
:105200008F4F9F4F2AE030E040E050E00E94543A38
:105210006901C2010E94A91A30E2E32E00E020E0F9
:10522000482FB201CE0101960E94C51A4ACF809143
:10523000F8039091F9034BCF0E946A1A882309F46E
:105240005BCF8091C303811708F056CF153009F06A
:1052500053CF00E027EA32E044E050E066E670E039
:1052600081ED92E047CF0A9660CF0E946A1A8823A8
:1052700009F48ECF153008F480CF8ACF0E94F11E3A
:105280009093F9038093F8036AE070E080E090E087
:105290000E94841480E00C94F8270F932091FA0365
:1052A0003091FB0381E02130310509F080E08093EB
:1052B00006012091F8033091F9033093E90320931C
:1052C000E80380913C01843009F058C04091FA0312
:1052D0005091FB03E09103010E2E000CFF0BE358ED
:1052E000FD4F60816403C001659F900D1124820F02
:1052F000931F9093F9038093F8038091EE03882322
:1053000059F000E027EA32E046E050E070E060E06B
:1053100087E091E00E942F2180913A0128E08202EB
:10532000C0011124FC01E65EFE4F408151812281C3
:1053300033816091F8037091F90326173707C0F5A0
:105340005093F9034093F803865E9E4F2091F80333
:105350003091F903FC013583248381E08093FC03C1
:105360000E94F3146093FD037093FE038093FF0388
:105370009093000480E00F910C94F827E0911801BD
:105380006091FA037091FB03EE0FFF0BEB59FD4F99
:1053900040815181649FC001659F900D749F900D65
:1053A0001124820F931F9093F9038093F803B4CFD5
:1053B0006417750748F63093F9032093F803C4CFB8
:1053C0000E94F8270E94F4250E944C220E946F211F
:1053D00081E00E9454240C944B25AF92BF92CF924F
:1053E000DF92EF92FF920F931F93CF93DF93B82E2C
:1053F000C0913A0191E0C23009F090E08091A2059D
:10540000837C8093A20520918D05203409F4F7C098
:105410009093A50580919205909193050E94261D79
:105420000C2F0C2E000C110BC33009F0F2C084E0DD
:1054300080933C01E09138010E2E000CFF0BE358E5
:10544000FD4F8081082E000C990BC0913601D09140
:105450003701E0903401F090350100913201109154
:10546000330110938F0500938E05F0929105E09221
:1054700090059093950580939405C017D10708F483
:10548000C6C0EC16FD0608F4C2C00E94821D9091B1
:10549000D5052091980530919A058091D2054091CB
:1054A000990540FB87F930FB86F98F7D20FB84F955
:1054B000807F8093D2059093D30580E280938D0501
:1054C0008091A205807C83608093A2051092A5053F
:1054D00081E08093A6050E94D01D8091D4050E9492
:1054E0005C1C1092D605809181050E94D11382E147
:1054F00090E00E94011990E080E00E9401198FEF76
:1055000090E00E94011990E080E00E94011990E073
:1055100080E00E94011990E080E00E9401190E9441
:1055200087178BE097E20197F1F710929605D093D9
:105530009305C0939205CE010E94261DB80180E01C
:1055400094E10E94281CB70181E094E10E94281C8C
:1055500065E070E082E094E10E94281C1092EA036A
:105560008091A5010E944E2061E070E081E095E10C
:105570000E94281C609139016093E60370E082E08C
:1055800091E10E94281C8091660161E0811162E036
:1055900070E080E091E10E94281C80913A0198E03F
:1055A0008902F0011124E65EFE4F2481358130939B
:1055B000F9032093F80320913C019681243009F0EF
:1055C000CEC190930301823038F480911801853068
:1055D0001CF084E0809318018091F603811103C0D0
:1055E00081E00E94E029DF91CF911F910F91FF9000
:1055F000EF90DF90CF90BF90AF900C94311A8D7FD9
:105600008093A2051092A5059093A60503CFE8010B
:105610003CCFE3E0000F111FEA95E1F7F801E65EE9
:10562000FE4FE080F180C280D380C23041F460E35D
:10563000C62E65E7D62E7EEAE72E76E0F72EF80135
:10564000E65EFE4FC6810C2E000CDD0B8091EA0356
:10565000882309F4F6C01092EC031092EB03B1100A
:105660000E94FD1E8091D1059091540190FB84F918
:105670008093D1050E94B11C80913C01B090C9017A
:10568000B394833011F0B0903C0190E080E0C730DB
:10569000D1053CF4FE01EE0FFF1FEB59FD4F808159
:1056A0009181F801E65EFE4F04811581F0928F052D
:1056B000E0928E05D0929105C09290059093950549
:1056C000809394050E151F0508F4B9C0C016D106C5
:1056D00008F4B5C09091D505209198058091D20528
:1056E0003091990530FB87F98F7920FB84F9807F11
:1056F00081608093D2059093D30580E480938D05DB
:105700008091A205807C81608093A2051092A505FE
:1057100081E08093A6050E94D01D8091D4050E944F
:105720005C1CB092D60582E0809396051093930599
:1057300000939205C8010E94261D0E94F21C8091D0
:10574000D1059091540190FB84F98093D1050E947A
:10575000B11C91E080915D01813009F490E080916D
:10576000D10590FB87F98093D1050E94B11C8091EF
:105770005D0190E0811193E08091D105807F892BBC
:105780008093D1050E94B11C60914B0170E082E0D2
:1057900093E30E94281C80913C0194E0833069F0DF
:1057A000E09105018E2FEE0F990BFC01EE0FFF1F0C
:1057B000E80FF91FEB56FD4F90819F708091D00547
:1057C000807F892B8093D0050E94B11C0E94651EAA
:1057D0008091D10590918A0190FB85F98093D10544
:1057E0000E94B11C0E94261E80916F0194EF980FB9
:1057F0009F3468F48093970524E531E0829FB001DF
:10580000839F700D112483E091E30E94281CB7014F
:1058100080E094E30E94281CB60181E094E30E949A
:10582000281C61E070E0C730D10534F4CC0FDD1FD7
:10583000CB59DD4F6881798182E094E3ACCE87015A
:1058400049CF10923C0190E080E0C730D1053CF494
:10585000FE01EE0FFF1FEB59FD4F80819181F80192
:10586000E65EFE4FA480B580F0928F05E0928E0533
:10587000D0929105C09290059093950580939405E0
:10588000AE14BF0408F469C0CA14DB0408F465C090
:10589000809196058130D1F10E94821D9091D505AD
:1058A000209198058091D2053091990530FB87F9B8
:1058B0008F7920FB84F9807F81608093D20590935B
:1058C000D30580E480938D058091A205807C816062
:1058D0008093A2051092A50581E08093A6050E9401
:1058E000D01D8091970594EF980F9F3458F424E5CC
:1058F00031E0829FB001839F700D112483E091E31A
:105900000E94281C8091D4050E945C1C1092D60530
:1059100081E080939605B0929305A0929205C5010F
:105920000E94261D60914B0170E082E093E30E948B
:10593000281CF801E65EFE4FE781E09304018E2FFC
:10594000EE0F990BFC01EE0FFF1FE80FF91FE05857
:10595000FD4F80810E949E1D45CF570199CF9093A6
:10596000180131CE282F41E060E089EC91E00E94DF
:10597000DE1980913C01833019F481E00C94ED290B
:105980000895282F41E060E08DE591E00E94DE1946
:105990000E946A1A8823F9F091E080915D018130BC
:1059A00009F490E08091D10590FB87F98093D105AF
:1059B0000E94B11C80915D0193E0811101C090E0D3
:1059C0008091D105807F892B8093D1050E94B11CE5
:1059D00081E00C94ED290895282F41E060E084E5F2
:1059E00091E00E94DE190E946A1A882369F0809172
:1059F000D1059091540190FB84F98093D1050E94C8
:105A0000B11C81E00C94ED290895FF920F931F9330
:105A1000CF93DF93F82E0091F8031091F9030E94C1
:105A20006A1A882351F08091EB039091EC0368EEA1
:105A300073E00E941E3A060F171FEFE3F2E0DF014A
:105A4000F11029C09496CD91DC919597C017D1079C
:105A500038F580913A01823061F5209751F1D09369
:105A6000F903C093F8031092EC031092EB030E9429
:105A70006A1A81110E94651ECE010E94261D0E9495
:105A8000261E80E00E94F827DF91CF911F910F9191
:105A9000FF900C94C325C081D1810C171D07C8F25B
:105AA0003296129742E0E536F40751F6D0E0C0E0B6
:105AB000D0CF90913C01E8E08E0290011124943007
:105AC00079F4265E3E4F90910301F9019683FF2001
:105AD00009F444C083304CF48F5F80933A0107C0CF
:105AE00090911801265E3E4FF0CF10923A018091BE
:105AF000F703882369F01092F70300E027EA32E009
:105B000046E050E070E060E087E091E00E942F21E5
:105B10008091EE03882389F080913C01843069F004
:105B20001092EE0300E027EA32E046E050E070E039
:105B300060E087E091E00E942F211092EC03109228
:105B4000EB030E946A1A81110E94651E80E0DF91BA
:105B5000CF911F910F91FF900C94ED29181614F41A
:105B60008150BBCF83E0B9CFCF93C82F83708330F0
:105B700001F58091F60381111CC0CB30D1F0C33008
:105B800011F41092C2038091C20391E0980F909398
:105B9000C203811109C080913A01683069F48330F1
:105BA0001CF481E00E94052D8091C20381708093D6
:105BB000C2038C2FCF9108958823B1F380E0F2CFF8
:105BC0000E94883A85ED8093BC008091B904909141
:105BD000BA04A091BB04B091BC040796A11DB11DED
:105BE00023E0B695A795979587952A95D1F72091AB
:105BF000BC0024FD03C01092B70408954091B9047D
:105C00005091BA046091BB047091BC04452B462BA3
:105C1000472B69F30097A105B10541F02AE22A95C7
:105C2000F1F700C00197A109B109E1CF8091B80453
:105C30000C9466171F93CF93DF93EC01162F0E94ED
:105C4000F439181739F0612FCE01DF91CF911F91F0
:105C50000C94FC39DF91CF911F910895FF920F931F
:105C60001F93CF93DF9366E788EE93E00E941A2E8E
:105C70006BEE90E080E00E941A2E6091EF036111BC
:105C800002C06091D40581E090E00E941A2E6091DC
:105C90003A0182E090E00E941A2E60913C0183E07C
:105CA00090E00E941A2E6091EC0384E090E00E9444
:105CB0001A2E6091EB0385E090E00E941A2E60910D
:105CC000030186E090E00E941A2E6091190187E09E
:105CD00090E00E941A2E6091050188E090E00E94F9
:105CE0001A2E0AE111E0C9E0D0E0F12CF80165813B
:105CF000CE010E941A2EF8016481CE0101960E9405
:105D00001A2EF8016681F3E0FF1619F067300CF0E7
:105D100060E0CE0102960E941A2EF8016781CE0142
:105D200003960E941A2EF394085F1F4F2496F4E006
:105D3000FF12DCCF0DE311E0C9E1D0E0F80165818D
:105D4000CE010E941A2E075F1F4F2196C932D1053E
:105D5000A9F7DF91CF911F910F91FF9008950C94B7
:105D6000F4391F920F920FB60F9211242F933F9385
:105D70008F939F93AF93BF93809150049091510460
:105D8000A0915204B091530430914F0423E0230FAB
:105D90002D3758F50196A11DB11D20934F04809316
:105DA000500490935104A0935204B09353048091F3
:105DB000540490915504A0915604B0915704019653
:105DC000A11DB11D8093540490935504A0935604D3
:105DD000B0935704BF91AF919F918F913F912F91B5
:105DE0000F900FBE0F901F90189526E8230F029674
:105DF000A11DB11DD2CF1F920F920FB60F92112489
:105E00002F933F934F935F936F937F938F939F93C2
:105E1000AF93BF93EF93FF93E091D001F091D10145
:105E20000995FF91EF91BF91AF919F918F917F91D4
:105E30006F915F914F913F912F910F900FBE0F90F7
:105E40001F9018951F920F920FB60F9211242F9347
:105E50003F934F935F936F937F938F939F93AF93F2
:105E6000BF93EF93FF93E091CE01F091CF0109959D
:105E7000FF91EF91BF91AF919F918F917F916F9122
:105E80005F914F913F912F910F900FBE0F901F90F8
:105E900018951F920F920FB60F9211242F933F93D4
:105EA0004F935F936F937F938F939F93AF93BF9322
:105EB000EF93FF938091B900887F803609F44AC040
:105EC000F0F5883209F4A7C018F5803109F49BC0B9
:105ED000B8F4882309F4F9C0883009F494C0FF911C
:105EE000EF91BF91AF919F918F917F916F915F9152
:105EF0004F913F912F910F900FBE0F901F901895CB
:105F0000883109F488C0803251F78093B50414C0F9
:105F1000803409F49DC040F48033B9F38833F9F636
:105F20008093B50485ECB0C0803509F485C0883510
:105F300009F496C0883499F60E94E22DD0CF8839B2
:105F400009F48CC038F5883729F050F4883611F000
:105F5000803729F683E08093B70410924C0457C031
:105F6000883809F47BC0803919F0803809F0B7CF40
:105F700080914C04803208F071C0E0914C0481E0C3
:105F80008E0F80934C048091BB00F0E0E45DFB4FEA
:105F900080833DC0803B39F0E0F4803A09F479C059
:105FA000883A09F09CCF84E08093B70410922B04C8
:105FB00010922A04E0918D04F0918E04099580914D
:105FC0002A0481110FC081E080932A0410920A04F0
:105FD00009C0803C09F4A6CF883C09F4A3CF883BD4
:105FE00009F07DCFE0912B0481E08E0F80932B048C
:105FF000F0E0E65FFB4F80818093BB0090912B0423
:1060000080912A0429C0809192048093BB0085EC82
:106010008093BC0064CF9091B4048091B30498172E
:1060200058F5E091B40481E08E0F8093B404F0E061
:10603000ED56FB4F8081E9CFE091B40481E08E0FF3
:106040008093B4048091BB00F0E0ED56FB4F808359
:106050009091B4048091B3049817C8F285E8D8CF22
:10606000E091B40481E08E0F8093B4048091BB0072
:10607000F0E0ED56FB4F80838091B60481115CCF38
:1060800081E08093910484EA8093BC001092B7046D
:1060900026CF85EC8093BC001092B70480914C040D
:1060A000803230F4E0914C04F0E0E45DFB4F10826C
:1060B00060914C0470E0E0918B04F0918C048CE2D0
:1060C00094E0099510924C040ACF1092B50434CF95
:1060D000FC016830A0F49AB121E030E0062E01C046
:1060E000220F0A94EAF7822F809589238AB98BB10F
:1060F000282B2BB9660F660F1082618308956E30CE
:1061000099F084B1262F2850330BA90121E030E00B
:1061100001C0220F4A95EAF7922F9095982394B9DF
:1061200095B1292B25B9E6CF3898409AE3CFE1EE17
:10613000F4E01382128288EE93E0A0E0B0E0848362
:106140009583A683B78386EB92E091838083E1EF0A
:10615000F5E01382128286E29BE19093F40480932F
:10616000F30481E29BE19093F2048093F10486EFC3
:1061700098E19093F0048093EF048EE698E1909379
:10618000EE048093ED0488EC92E0918380830E947A
:10619000F3146093ED057093EE058093EF059093F3
:1061A000F00565E08BEE95E00E94683068E089EECE
:1061B00095E00E94683069E087EE95E00E946830C3
:1061C00066E085EE95E00E94683067E083EE95E03A
:1061D0000E9468306EE081EE95E00E9468306BE0CE
:1061E0008FED95E00E9468306AE08DED95E00E94A9
:1061F000683064E08BED95E00E946830E8EDF5E0F2
:1062000082E0818383E08283529853985A9A5B9A02
:10621000108210927F051092800581E190E09093AA
:106220008205809381058EE190E0909384058093B0
:1062300083058AE090E0909386058093850580E44D
:106240009FE1A0E0B0E08093870590938805A0933C
:106250008905B0938A058FEF8093960594E2909319
:10626000970591E0909398051092990510929A05E0
:1062700020E030E830939C0520939B0521E030E03E
:1062800030939E0520939D0510929F0590E2909378
:10629000D40595E09093D5058093D7051092D60547
:1062A0000895789484B5826084BD84B5816084BD8E
:1062B00085B5826085BD85B5816085BD80916E00A4
:1062C000816080936E0010928100809181008260D5
:1062D0008093810080918100816080938100809112
:1062E00080008160809380008091B1008460809301
:1062F000B1008091B00081608093B00080917A00FD
:10630000846080937A0080917A00826080937A0022
:1063100080917A00816080937A0080917A00806811
:1063200080937A001092C100259A52985A9A5398F5
:106330005B9A0E94021421E08D3291400CF420E01F
:106340002093E50310925C0410925B0480E8809334
:10635000D20188E08093D301E091F304F091F4043A
:1063600009950E948915C5EFD6E2EBEFEE2EE6E225
:10637000FE2EFE011491812F0E945715811107C036
:106380000E9452150E948915812F0E94571521964F
:10639000EC16FD0671F70E9452150E94B8150E9476
:1063A00089158FEA0E9457150E94521587EA92E0DC
:1063B0000E94DD13309905C30E942E2E87EF92E0D4
:1063C0000E941D2162E080E00E948E15C0E186E0FF
:1063D00093E00E941D216CE370E080E090E00E9459
:1063E0008414C150A1F70E94B81520E43AE130931B
:1063F000CF012093CE01809169008C7F81608093D2
:106400006900E89A3093D1012093D001809169000E
:10641000837F846080936900E99A8CE080938C0587
:106420000E94B7140E944F1781E10E94D1130E946D
:1064300087178111FDC281E190E0909382058093DE
:1064400081050E944F178CE080938C05109299056E
:1064500010929A0585E08093D50591E19093D2053D
:106460008093D30591E09093980580E480938D0507
:106470008091A205807C81608093A2051092A50581
:106480009093A6058091D70587FD07C061E00E9423
:1064900013148BEA94E00197F1F70E94B7140E945D
:1064A000D01D8EE10E945C1C0E94101C8091810511
:1064B0000E94D11380E190E00E9401190E94871789
:1064C00000EC15E00E94101C69E070E080918105ED
:1064D000909182050E943A1BC7EBD5E081EE94E0D3
:1064E0000E94801889930C171D07C1F78091B7058A
:1064F00086FDE8CF6AEF70E080E090E00E948414AF
:1065000000E027EA32E050E040E070E060E088E43C
:1065100093E00E942F2164EF71E080E090E00E9400
:1065200084140E94B81588EE93E00E94AF2E86373F
:1065300009F0A9C290E080E00E94AF2E8B3E09F0E6
:10654000A2C281E090E00E94AF2E8093000182E021
:1065500090E00E94AF2E80933A0183E090E00E9489
:10656000AF2E80933C0184E090E00E94AF2EC82FB4
:1065700085E090E00E94AF2E9C2F9093EC038093D7
:10658000EB0386E090E00E94AF2E8093030187E04A
:1065900090E00E94AF2E8093190188E090E00E9465
:1065A000AF2E809305010AE111E0C9E0D0E0CE01F1
:1065B0000E94AF2EF82ECE0101960E94AF2E9F2D85
:1065C000F80195838483CE0102960E94AF2EF801D4
:1065D0008683CE0103960E94AF2EF801878324960E
:1065E000085F1F4FC931D10511F70DE311E0CE014E
:1065F0000E94AF2EF80185832196075F1F4FC93295
:10660000D105A9F7C0917801CC0F0E94891581E8C6
:106610000E9457158C2F0E9457150E9452152091E9
:106620003A01F8E02F02C0011124FC01E65EFE4FA2
:10663000448155815093F9034093F8035093E90343
:106640004093E803233009F0FDC1209138012093E5
:106650000301865E9E4FFC01C7818091180187303F
:1066600014F0109218010E946A1A882309F4EEC1EE
:106670000E94FD1EE09105018E2FEE0F990BFC018B
:10668000EE0FFF1FE80FF91FEB56FD4F90819F7033
:106690008091D005807F892B8093D0050E94B11C0A
:1066A0000E94F21C80E00E94ED29F89480E880931B
:1066B000610080919C0180936100789480E00E9449
:1066C000ED290E94F11E9093E9038093E8039093D3
:1066D000F9038093F803809100010E945C1C0E94E2
:1066E000B81580E00E94E0296624639458EEC52E18
:1066F00053E0D52E0E94F3141B012C018090FD0362
:106700009090FE03A090FF03B09000048091FC03E2
:106710008823E9F00E946A1A811119C028183908E3
:106720004A085B088091FA039091FB03F6E42F1668
:1067300031044104510408F4A9C1892B41F480912A
:10674000F8039091F9030E94261D1092FC030E9409
:10675000F314681979098A099B09683E7340810519
:10676000910578F00E94D2228091F703882331F0BE
:106770008091F603811102C00E94B02180E00E9446
:10678000542420900104309002044090030450905F
:106790000404211431044104510469F00E94F314EB
:1067A0006219730984099509693B7B40810591054C
:1067B00010F00E94BF198091FA039091FB03892B7E
:1067C00009F06EC16AED79E18BEE95E00E94061941
:1067D000813071F48091F60381110AC080913C01EF
:1067E000833031F06FE671E281EF93E00E94312651
:1067F00064EB7DE289EE95E00E940619813061F438
:106800008091F603811121C40E94E92764EF75E2AB
:1068100080EF93E00E94312664EB7DE287EE95E005
:106820000E9406198130E9F48091F603811102C0BB
:106830000E94BF198091F60386258093F6030E947B
:10684000B8158091F603882309F41AC4F1E0F09397
:10685000CD010E9470261092F4031092F5030E945D
:10686000AF276EE975E285EE95E00E94061981304A
:1068700071F48091F60381110AC08091EF038111B8
:1068800006C06BE475E283EF93E00E9431266EE967
:1068900075E283EE95E00E940619813099F48091AB
:1068A000F30381110FC09091D4058091EF039923D8
:1068B00009F4ECC38111EDC39093EF030E945C1CBB
:1068C0000E944B256AED79E181EE95E00E94061960
:1068D000813049F49091F003992309F4DFC31092B9
:1068E000F0030E94F42570E060E08FED95E00E94D7
:1068F0000619813009F0FAC480913B019091F603AA
:10690000992311F081110DC0862580933B018823C6
:1069100009F4E8C40E9489158FEA0E9457150E9465
:10692000521570E060E08DED95E00E94061981300F
:1069300009F0ECC48091F603811108C06CE472E2A6
:1069400082EF93E00E9431260E94E9276AED79E107
:106950008BED95E00E940619813009F0F2C090910C
:10696000F6039111EEC090913C01943009F41CC5DE
:10697000C0913A01E090F803F090F90388E0C80272
:10698000E0011124FE01E65EFE4FF582E482809173
:106990003C018093190180913C01813009F4D0C4FD
:1069A00008F4CAC4823009F4DFC4833009F4E4C4B3
:1069B00080911801C65EDE4F8E8380E00E94ED2933
:1069C000C0C001E027EA32E050E040E070E060E063
:1069D00088E093E00E942F21209101013091020173
:1069E00000E042E050E070E060E089E193E00E9466
:1069F0002F21209101013091020144E050E070E02C
:106A000060E087E293E00E942F2120910101309104
:106A1000020146E050E070E060E088E393E00E940D
:106A20002F2168EB7BE080E090E00E948414DBCCB7
:106A300083E60E94D1130E948717811102CD83E65D
:106A400090E0FBCC26812093180103CE80913C017D
:106A5000811110C0C09304010C2E000CDD0BFE014F
:106A6000EE0FFF1FEC0FFD1FE058FD4F80810E94CD
:106A70009E1D18CEC093E6036C2F70E082E091E17A
:106A80000E94281C0FCE0E942E2E0FCE892B09F4B7
:106A90005ECE0E944D291092FB031092FA032ACE7B
:106AA0008091010490910204A0910304B091040428
:106AB000892B8A2B8B2B51F00E94F31460930104D5
:106AC0007093020480930304909304048091F6036E
:106AD000882309F490C01091F5038091F4031111FB
:106AE0006EC06091FA037091FB03680F2091CD0195
:106AF0002150922F990F920F990F75E0790F7031F5
:106B000008F07FE0462F062E000C550BE6E02E9F86
:106B100090011124421753070CF048C07093F403FE
:106B200061E00E949B2661E08091F4030E949B2615
:106B30001092FB031092FA030E94311A112309F4F8
:106B400041CE2091F8033091F9038091E8039091B0
:106B5000E9032817390709F4CDCD0E94F3140091F9
:106B6000ED051091EE052091EF053091F005601BC9
:106B7000710B820B930B613177428105910508F40B
:106B8000B9CD0E942E2E0E94F3146093ED057093F0
:106B9000EE058093EF059093F0058091F8039091B6
:106BA000F9039093E9038093E803A4CD74171506C5
:106BB0001CF49093F403B4CF6093F403B1CF20910D
:106BC000FA033091FB0399E08902F0011124E35CA0
:106BD000FE4F0780F085E02D822F099560E08091BF
:106BE000F4030E949B2664E670E080E090E00E943F
:106BF000841410E09DCF1091F303112339F080919C
:106C0000FA039091FB030E948125F3CF8091F20358
:106C1000882309F4CEC0C091FA03D091FB03809180
:106C20003C018430A1F580910301C13039F58F5FBB
:106C3000833034F11092030120910301E22F022EE0
:106C4000000CFF0BE358FD4F8081082E000C990BC0
:106C50009093950580939405E0913A0138E0E30222
:106C6000F0011124E65EFE4F268365E070E082E0CD
:106C700094E10E94281C0E944C225ACF8150D8CF08
:106C800087FD03C080930301D7CF82E0FBCF8091C3
:106C90001801C13009F04AC08F5F80931801D0916C
:106CA00018010E94751A2D2FDD0F330B82179307E1
:106CB0000CF03EC0109218010E946A1A81116EC039
:106CC000E0911801EE0FFF0BEB59FD4F8081918190
:106CD000909395058093940580911801E0913A0175
:106CE00098E0E902F0011124E65EFE4F86830E94DF
:106CF0006A1A8111C0CFE0913A0128E0E202F00166
:106D00001124E65EFE4F8681082E000C990B61E08F
:106D100070E0873091053CF4880F991FFC01EB5916
:106D2000FD4F6081718182E094E3A3CF8150B5CFA4
:106D30008091180187FF05C00E94751A8093180181
:106D4000BBCF0E946A1A882369F0809118018430B1
:106D50004CF08091180187302CF483E0C13071F73A
:106D600087E0ECCF80913A01823008F0A5CF809186
:106D70001801C13049F485300CF49ECF8091180180
:106D800087300CF099CFECCF85300CF495CF809103
:106D9000180187300CF090CF84E0D0CF0E946A1A9F
:106DA000882309F4A4CF8091180187300CF488CF90
:106DB0009ECF1091F103112309F45FC0E090FA0314
:106DC000F090FB030E946A1A882311F12E2D45E0F2
:106DD00060E085E091E00E94DE19E09105018E2FD0
:106DE000EE0F990BFC01EE0FFF1FE80FF91FEB569A
:106DF000FD4F90819F708091D005807F892B80937B
:106E0000D0050E94B11C0E94F21C0E946F21F1CE9D
:106E100080913C01C0913A0138E0C302E0011124A5
:106E20002E2D811119C046E060E084E091E00E94BF
:106E3000DE19E0910401C65EDE4FEF838E2FEE0F68
:106E4000990BFC01EE0FFF1FE80FF91FE058FD4FF3
:106E500080810E949E1DD9CF44E060E086EE93E0E1
:106E60000E94DE196091E603C65EDE4F6F8370E01C
:106E700082E091E10E94281CC8CF8091F003882312
:106E800061F08091FA039091FB03019721F481E076
:106E90000E94052D4DCE80E0FBCF0E946A1A182F6C
:106EA000882309F4CEC08091FA039091FB030197E7
:106EB00009F090C00E947F1AC091EB03D091EC03BF
:106EC000C80FD91F2091F8033091F903C1388EE320
:106ED000D8070CF485C0CE0160E87EE30E941E3A1C
:106EE000E82F492F80E89EE3689F4001699F900C3E
:106EF000789F900C1124C401B6010E941E3A620FC3
:106F0000731F7093F9036093F803CE2FD42FD0939F
:106F1000EC03C093EB030E94651EE0903A010E2C37
:106F2000000CFF08892871F08091F8039091F90313
:106F30000E94261D0E94261E0E94F11E9093F903B6
:106F40008093F803CE01B6010E941E3A8090F803A8
:106F50009090F903860E971EE70183E0CC0FDD1FAA
:106F60008A95E1F79E01265E3E4F7901F9019582EF
:106F700084820E94F3146093FD037093FE03809358
:106F8000FF03909300041092E9031092E803F701C5
:106F900082819381208131818815990508F045C04F
:106FA0003093F9032093F8038091F8039091F9034B
:106FB000C65EDE4F9D838C830E94261D1092EC03DB
:106FC0001092EB030E94651E81E00E94F8270E9448
:106FD000F425AECD0E947F1A9195819591096CCFD1
:106FE000912C812CC03891ECD9070CF090CF8827D8
:106FF00099278C1B9D0B60E87EE30E941E3AE0E817
:10700000FEE36E9F40016F9F900C7E9F900C1124B9
:10701000C401B6010E941E3A261B370B3093F903B8
:107020002093F803C80DD91D72CF8216930620F065
:1070300080E00E94F8277CCD9093F9038093F803B9
:10704000B3CF0E944D2911E073CD8091CD018F5FA8
:1070500084300CF081E08093CD01082E000C990B58
:107060000197982F990F890F880F8093F40310923E
:10707000F5030E94B8150E9470260E94AF27CCCB62
:107080000E942E2E80E00E94E029EBCB882309F499
:1070900017CC0E945C1C1092EF0312CC9091F2036B
:1070A000992329F01092F2030E944C221CCC90915B
:1070B000F103992329F01092F1030E946F2113CC60
:1070C0009091F303992329F01092F3030E944B252A
:1070D0000ACC9091F603992359F09091F5038927F2
:1070E0008093F50361E08091F4030E949B26FBCB23
:1070F0009091EE03992319F08093ED03F4CB0E9455
:107100006A1A8111C7C08091C001882309F4C2C0E6
:1071100080913C01843009F0C6C063E070E081E0FA
:1071200090E40E94281C2091060180919205909184
:107130009305222309F4C3C0209190053091910555
:107140008217930708F4B4C080918E0590918F0543
:107150009093930580939205809192059091930569
:107160000E94261D1092E703D09106010E94F3149D
:107170001B012C0180919605823009F47BC080911F
:107180008D05C1E2803209F0C1E40E94101CD0FBE1
:1071900073F8272D2870722E809181050E94D113DB
:1071A0006C2F81EE94E00E94C718672D81EE94E069
:1071B0000E94C718C134E9F4C1E080919205909112
:1071C00093058930974008F4C0E060E081EE94E0D8
:1071D0000E94C71860E081EE94E00E94C71860E04A
:1071E00081EE94E00E94C7186C2F81EE94E00E941B
:1071F000C7180E94871768E770E080E090E00E945F
:107200008414609183057091840590E080E00E9471
:10721000841480E00E94A21E609183057091840511
:1072200090E080E00E9484149091B1058091B205B5
:1072300080939205909393050E943E290E94291AFB
:10724000811118C08091B0058178A1F40E94F314D7
:1072500062197309840995090091870510918805C1
:107260002091890530918A0560177107820793077D
:1072700008F485CF0E94F11E9093F9038093F803E0
:1072800081E00E94E02970E060E081E090E40E94EB
:10729000281C29CB6CE472E282EF93E00E94312635
:1072A0000E94E92720CB80913C0181111CCB35CF76
:1072B0002091940530919505820F931F49CF20911D
:1072C0008E0530918F052817390728F08091900599
:1072D000909191053DCF2091940530919505821BA9
:1072E000930B36CF0E9489158EEA17CB873009F0B1
:1072F00018CB8091F603811114CB0E946A1A88235F
:1073000009F40FCB81E00E94C12C0BCB8B3009F02C
:107310001DCB8091F603811119CB8091F70386254F
:107320008093F703882329F01092EE030E94B02186
:107330000DCB0E94D5270ACB0E94FD1E1092FC03A4
:1073400080913C018F5F80933C01FE01E65EFE4F21
:107350008091EB039091EC03B6010E941E3A6E0DF2
:107360007F1D7583648324CB80913C018F5F809364
:107370003C011092F103ECCF10923C011092EA0311
:1073800080911801873014F0109218018091EB035E
:107390009091EC03B6010E941E3AE60EF71EF092A1
:1073A000F903E092F80304CB9091EE0389278093D0
:1073B000EE038823B1F01092F70300E027EA32E0F1
:1073C00046E050E070E060E087E091E00E942F210D
:1073D00080918D05803211F40E94F31F0E94D22209
:1073E000B0CB0E94D527ADCBF999FECF92BD81BD20
:1073F000F89A992780B50895262FF999FECF1FBADC
:1074000092BD81BD20BD0FB6F894FA9AF99A0FBECD
:1074100001960895AA1BBB1B51E107C0AA1FBB1F01
:10742000A617B70710F0A61BB70B881F991F5A9510
:10743000A9F780959095BC01CD01089597FB072E83
:1074400016F4009407D077FD09D00E940A3A07FC91
:1074500005D03EF4909581959F4F08957095619564
:107460007F4F0895A1E21A2EAA1BBB1BFD010DC080
:10747000AA1FBB1FEE1FFF1FA217B307E407F507E4
:1074800020F0A21BB30BE40BF50B661F771F881FC0
:10749000991F1A9469F760957095809590959B0156
:1074A000AC01BD01CF010895052E97FB1EF4009499
:1074B0000E946B3A57FD07D00E94323A07FC03D076
:1074C0004EF40C946B3A50954095309521953F4F72
:1074D0004F4F5F4F089590958095709561957F4FC0
:1074E0008F4F9F4F0895EE0FFF1F0590F491E02DF1
:1074F0000994A29FB001B39FC001A39F700D811D8D
:107500001124911DB29F700D811D1124911D0895AC
:0E75100081E090E0F8940C948D3AF894FFCF4F
:10751E0019A7020104040120202020202020202071
:10752E0020202020202020000304950008022C019A
:10753E0000040802AE06C4050304AE063075AE069E
:10754E0000042E22302A2E2201000101044154543F
:10755E00000000005C1E534D20000000019E1C53D5
:10756E00564300000102EC2C53796E00000002C15C
:10757E002C44654500000102681C41564300002E54
:10758E00017F1C53637200005001111A53572000E3
:10759E000000020A1A53534D00000102DC1C434F37
:1075AE004600000003191D43505500000002F91952
:1075BE0052445300000101AD2042464F000000012D
:1075CE00BD20556E7400000102F21953636E000067
:1075DE000102EB1943572000000002B22C01FF14E8
:1075EE00FF148004830264006C025F005C025A0088
:1075FE00450250003D023C002E0228001E021400DF
:10760E00F7010F00F0010500E80100000002040080
:10761E000300011003020000030201000600040033
:10762E00060500200605040068000E032E39000032
:10763E0000000059035D036103650369036D037068
:10764E00037303D20276037B03800385038A03AEA2
:10765E0006AC0D9411E015901A201C34211027C091
:10766E002B5834B036983A30435046085298533A15
:10767E00615866606D0100050009000A0032006461
:10768E0000E8030A00190032006400F401050A64E0
:10769E00048F03059403039903069E0302A30301BB
:1076AE00A80300AD0304B203058F0300B70301BCAA
:1076BE000302A30303A80360020802207E00000059
:1076CE00000000000000C7189A18371B7018931896
:1076DE008018711800000000271A0015371B361B82
:1076EE0020202020005374703A00434200530020A3
:1076FE00202053455454494E47532020002F2F2FFE
:10770E002F2F2F2F2F2F002020454550524F4D2029
:10771E005245534554002D00544F50544543482074
:10772E005245434549564552002020203D3D4532A5
:10773E003558435A3D3D004669726D77617265203A
:10774E00562E312E302E3600206E727368616D63A8
:10775E006C75622E636F6D00496E697469616C6938
:10776E007A6174696F6E2E2E00414D20004C53428B
:10777E00005553420043572000464D20004C570001
:10778E004D57005357004155544F003131306B0067
:10779E002038346B002036306B002034306B0031D3
:1077AE002E306B00312E386B00322E306B00322EA5
:1077BE00356B00332E306B00342E306B00362E308E
:1077CE006B00302E356B00312E326B00322E326B49
:0277DE000000A9
:00000001FF
